:0400000022EF31F0CA
:1000080000C016F001C015F0E1CF17F0E2CF18F0EC
:100018009EAA6ED09DAA6CD0AECFCEF0ABA210D067
:10002800AB98010E00019925006E000E9A21016E11
:1000380000C099F001C09AF0AECFCEF0AB88CE6B7D
:10004800ABA40FD00001AB9E010E9925006E000EE7
:100058009A21016E00C099F001C09AF0AB8EAECF24
:10006800CEF00001CE510D0A04E11B50010A01E156
:1000780007D0C151000802E1C051620801E322D053
:10008800010ECC6F000ECD6FA00ECA25E16E050ED5
:10009800CB21E26EE66A9D9A6B96CAC0C0F0CBC0CF
:1000A800C1F0CA6BCB6BC151000802E1C0516308B3
:1000B80004E2020ECC6F000ECD6F9EAA02D0AECF26
:1000C800CEF016D0A00ECA25E16E050ECB21E26E49
:1000D800CEC0E6FFCAC0C0F0CBC0C1F0010ECA2531
:1000E800006E000ECB21016E00C0CAF001C0CBF03B
:1000F800F2A809D0F2A207D00001010EE36F000EAA
:10010800E46FF292F2989DA01ED09EA01CD0010E22
:100118000501575D006E000E5859016E00C057F575
:1001280001C058F5000E585D02E1010E575D06E268
:100138009D90CD90010E556F000E566F3C0ECF6E00
:10014800B00ECE6E9E9016C000F015C001F017C01C
:08015800E1FF18C0E2FF1100F5
:100160000B820BAEBAEF00F003680268016800680A
:080170000A360232FF0E1200F4
:0E017800026A016A006A086A036A000E120039
:100186000B840BAECEEF00F0010E036E026A016A1D
:0A019600006A0A360232FF0E120062
:0801A0000AAE029E000E1200DF
:0C01A80072B201D0FDD7ADC673FF12008B
:0E01B400ACB202D00000FCD7ADC6ADFF120009
:1001C2000CB023EF01F00CA2C9EF01F00E6A000E91
:1001D20002643AEF01F0F00E0214D8A405EF01F028
:1001E200023A01380F0B02260138F00B016E00387B
:1001F2000F0B01260038F00B006E08380F0B00269B
:100202000838F00B086E0E84D89002BE1EEF01F083
:1002120008360036013602360E2A02BE1EEF01F003
:1002220008360036013602360E2A02BE1EEF01F0F3
:1002320008360036013602360E2A0E500364BFEF2E
:1002420001F0035E0BBC08AEC4EF01F0D880800E53
:1002520008640030000E002201220222D8A0C4EF5E
:1002620001F0023201320032034AC9EF01F0C4EF59
:1002720001F001C002F000C001F008C000F0086AFD
:10028200000E0E86026471EF01F0F00E0214D8A483
:1002920059EF01F0023A01380F0B02260138F00B38
:1002A200016E00380F0B01260038F00B006E0E8431
:1002B200D89002BE1EEF01F00036013602360E2A39
:1002C20002BE1EEF01F00036013602360E2A02BED1
:1002D2001EEF01F00036013602360E2A1EEF01F043
:1002E20001C002F000C001F0006A000E0E960E88F6
:1002F20002649EEF01F0F00E0214D8A489EF01F01F
:10030200023A01380F0B02260138F00B016E0E84FF
:10031200D89002BE1EEF01F0013602360E2A02BE4E
:100322001EEF01F0013602360E2A02BE1EEF01F068
:10033200013602360E2A1EEF01F001C002F0016AF8
:10034200000E0E860264CEEF01F0F00E0214D8A465
:10035200ADEF01F0023A0E84D89002BE1EEF01F01A
:1003620002360E2A02BE1EEF01F002360E2A02BE2D
:100372001EEF01F002360E2A1EEF01F0010E0C6E86
:1003820001DFD1EF01F0020E0C6E09DFD1EF01F0B7
:10039200040E0C6EE4DED1EF01F0080E0C6EEBDE03
:0203A200120047
:1003A400086A080E0C6E003408360450085ED8B093
:0E03B40002D00826D89000360C2EF5D7120085
:1003C200025006180E6E086A096A0B6A0350076427
:1003D200D4EF02F006500A6E068E028E03500B6EA8
:1003E2000750036E000E0B6424EF02F00B50075E01
:1003F200D8B4C5EF02F0070E076493EF02F0075E70
:1004020000C008F001C000F002C001F0026A074E0D
:10041200C5EF02F0076468EF02F0075E00C008F063
:1004220001C000F0016A074EC5EF02F0076446EF13
:1004320002F0075E00C008F0006A074EC5EF02F046
:1004420007642DEF02F00AC002F005C001F004C0FB
:1004520000F0086AEEEF03F0030E076438EF02F0D3
:10046200075E08380F0B086E074EC5EF02F0D890F2
:100472000832074EC5EF02F0D8900832074EC5EF9A
:1004820002F0D8900832C5EF02F0030E076457EF6E
:1004920002F0075E08380F0B086E0038F00B0826D2
:1004A20000380F0B006E074EC5EF02F0D8900032F5
:1004B2000832074EC5EF02F0D89000320832074EDC
:1004C200C5EF02F0D89000320832C5EF02F0030EF9
:1004D20007647FEF02F0075E08380F0B086E0038E2
:1004E200F00B082600380F0B006E0138F00B0026C7
:1004F20001380F0B016E074EC5EF02F0D8900132A2
:1005020000320832074EC5EF02F0D89001320032B5
:100512000832074EC5EF02F0D8900132003208329D
:10052200C5EF02F0030E0764B0EF02F0075E083871
:100532000F0B086E0038F00B082600380F0B006E08
:100542000138F00B002601380F0B016E0238F00B58
:10055200012602380F0B026E074EC5EF02F0D8904B
:100562000232013200320832074EC5EF02F0D89053
:100572000232013200320832074EC5EF02F0D89043
:100582000232013200320832096A000E0EAEB9EFB1
:1005920003F0081E001E011E021E082A002201226C
:1005A2000222B9EF03F00750D8A4DAEF02F0EEEF1F
:1005B20003F0096A02C00AF0028E068E0750035C3D
:1005C200076ED8B4ACEF03F0070E07647AEF03F0BE
:1005D200075E0450096E0550046E0650056E066AE9
:1005E200074EACEF03F0070E07644FEF03F0075E10
:1005F2000450096E0550046E056A074EACEF03F015
:10060200070E07642DEF03F0075E0450096E046ABB
:10061200074EACEF03F0070E076414EF03F00AC0B5
:1006220002F0EEEF03F0030E07641FEF03F0075E24
:1006320009380F0B096E074EACEF03F0D890093260
:10064200074EACEF03F0D8900932074EACEF03F03F
:10065200D8900932ACEF03F0030E07643EEF03F0CB
:10066200075E09380F0B096E0438F00B09260438AF
:100672000F0B046E074EACEF03F0D8900432093230
:10068200074EACEF03F0D89004320932074EACEFBC
:1006920003F0D89004320932ACEF03F0030E076482
:1006A20066EF03F0075E09380F0B096E0438F00B92
:1006B200092604380F0B046E0538F00B04260538A2
:1006C2000F0B056E074EACEF03F0D89005320432E3
:1006D2000932074EACEF03F0D890053204320932EA
:1006E200074EACEF03F0D890053204320932ACEF7A
:1006F20003F0030E076497EF03F0075E09380F0B50
:10070200096E0438F00B092604380F0B046E053805
:10071200F00B042605380F0B056E0638F00B052684
:1007220006380F0B066E074EACEF03F0D890063278
:10073200053204320932074EACEF03F0D89006328C
:10074200053204320932074EACEF03F0D89006327C
:10075200053204320932086A000E0EAEB9EF03F018
:10076200091E041E051E061E092A0422052206224F
:100772000950082604500022055001220650022288
:100782000EBED0EF03F0D8A0DFEF03F00232013249
:1007920000320832033EDFEF03F0E9EF03F0D8B096
:1007A200E4EF03F0000E081E001E011E021E082ABE
:1007B2000022012202220A7EE4EF03F0010E0C6EF7
:1007C200FFDCF0EF03F0020E0C6EFADCF0EF03F048
:1007D200040E0C6EC4DCF0EF03F0000E0C6E12007F
:1007E2000134083609360450085E0550D8A0053C8D
:1007F200095E003601360F0E0C6E013408360936DA
:10080200045000A006D0085E0550D8A0053C095E41
:1008120005D008260550D8B0053C09260036013619
:100822000C2EEBD700B006D0045008260550D8B0E5
:08083200053C0926000012003C
:10083A000D6A086A0050D8B4000C04180A6E0ABE81
:10084A000D1E0B6A04AE02D0041E042A00AE02D0AA
:10085A00001E002A005004100A6E0ABE1FD004505F
:10086A00085E003600340836045008260036060EA4
:10087A000C6E00340836045000B0085E00A008264A
:10088A0000360C2EF6D700A008260BB015D00DAEF8
:10089A00000C001E002A081E082A000C04AE09D00B
:1008AA0000BE04D00050086E006AF1D7006A002A20
:1008BA00000C001E0B2AD3D7082A0450085CD8A4BF
:0E08CA00E6D7086A002A00AEE2D7FF0C120043
:1008D8000B800BAE78EF04F0026A0AAEFF0E026ED0
:0C08E800016E006E0A360232FF0E120094
:1008F400086A096A000E07620364FFEF04F00250FD
:1009040006180A6E075003267E0ED8A090EF04F056
:10091400035ED8B004EF05F094EF04F0035ED8A0B2
:1009240009EF05F0028E068E02C00EF001C00BF036
:1009340000C00DF000500402F4CF0CF00150050289
:10094400F4CF00F0F3CF08F00402F3500C26F45077
:100954000822000E00220D500502F3500C26F4501C
:100964000822000E002202500402F3500826F4501C
:10097400002202500502016A000E0122F3500026F3
:10098400F45001220D500602F3500826F4500022C0
:10099400026A000E012202220B500602F3500026C6
:1009A400F4500122000E02220E500602F3500126DA
:1009B400F450022202BEE7EF04F008360036013696
:1009C40002360306D8B409EF05F0FAEF04F0D88034
:1009D400800E08640030000E002201220222D8A0FA
:1009E400FAEF04F0023201320032034A04EF05F058
:1009F4000AAE029E000E0CEF05F0010EBCEC00F0F6
:100A04000CEF05F0020EB0EC00F00CEF05F0040E54
:060A1400C3EC00F012002B
:080A1A000B6A0B86FF0E1200AF
:100A2200F250026EF29E0500FF6A0150FE6E005007
:080A3200FD6E02BEF28E1200FF
:100A3A00C7B409D01F0EC514016E0150000A03E1A4
:0A0A4A00010E006E01D0006A1200D8
:100A540003500718D8A43EEF05F002500618D8A496
:100A64003EEF05F001500518D8A43EEF05F0005004
:0E0A74000418D8B4D8841200D89412001200CE
:100A82000450000A08E10550000A05E1FF0E006E5D
:100A92007F0E016E57D00D6A096A086A0150001074
:100AA200D8B4000C015005180A6E0ABE0D1E0B6A5E
:100AB20005AE05D0041E051E042AD8B4052A01AECF
:100AC20005D0001E011E002AD8B4012A01500510CB
:100AD2000A6E0ABE10D084DE0BB020D00DAE000C20
:100AE200001E011E002AD8B4012A081E091E082A67
:100AF200D8B4092A000C05AE0DD001BE07D00150B2
:100B0200096E0050086E016A006AE8D7016A006A3D
:100B1200002A000C011E001E0B2ADDD7082AD8B4B9
:100B2200092A0450085CD8A4D9D70550095CD8A476
:100B3200D5D7096A086A002AD8B4012A01AECED7ED
:060B42000000FF0C120090
:100B48000B6A0C6A0A6A086A0350D8B42CEF06F0DC
:100B5800028E9E0E035E03BEB7EF05F0D8B4B7EF62
:100B680005F01CEF06F0036C080E035CD8A0E9EF53
:100B780005F0036E083600C008F001C000F002C09E
:100B880001F0026A080E035CD8A0E9EF05F0036ED5
:100B9800083600C008F001C000F0016A080E035CC6
:100BA800D8A0E9EF05F0036E083600C008F0006A27
:100BB800080E035CD8A0E9EF05F0036E0836086A52
:100BC8000350D8A4D890F5EF05F00350D8B4F5EF4A
:100BD80005F0D8900232013200320832032EEDEFD0
:100BE80005F00BBC08A006EF06F0D8A006EF06F04B
:100BF800082AD8B4002AD8B4012AD8B4022A02BED6
:100C080030EF06F00AAE2CEF06F0021E011E001EA1
:100C1800081E082AD8B4002AD8B4012AD8B4022A4F
:100C28002CEF06F0026A016A006A086A2CEF06F0E7
:100C38000B800BAE35EF06F0026A0AAE35EF06F010
:100C4800026E016E006E086E0A36023235EF06F04B
:100C5800000E0C6A36EF06F0010E0C6E39DE36EF28
:100C680006F0FF0E0250036E0150026E0050016E36
:060C78000850006E12009E
:100C7E000050086E0150006E0250016E0350026E5D
:100C8E00036A0B6A0C6A9E0E036E0A6A020E0C6EE3
:060C9E00E1EC00F0120081
:080CA400067EE1EC01F01200F4
:100CAC008B90A7C604F0026A036A800E0318006ECC
:100CBC00800E005C02E1080E025C1FE2800E041440
:100CCC00016E0150800A02E18B8401D08B941A0EC4
:100CDC000D6E0D2EFED70000043604908B801A0E7C
:100CEC000D6E0D2EFED700008B901A0E0D6E0D2E74
:0C0CFC00FED70000024A032AD8D71200DD
:100D08000450000A12E10550000A0FE10650000ADB
:100D18000CE10750000A09E1FF0E006EFF0E016E9C
:100D28007F0E026EFF0E036EA7D0086A096A07508D
:100D3800D8B42FEF07F00350D8B433EF07F00250C0
:100D480006180A6E028E068E0E6A02C008F001C0EE
:100D58000CF000C00DF004500D5E0550D8A0053C05
:100D68000C5E0650D8A0063C085E086A0C6A0D6A3C
:100D7800D8A0C6EF06F0D89002320132003208320D
:100D8800010E0E6E0750035ED8A0D3EF06F07E0E5C
:100D98000E240326D8B038EF07F0D9EF06F07E0E00
:100DA8000E240326D8A03DEF07F0180E0B6E0D3663
:100DB8000C3608360036013602360E360450005E10
:100DC8000550D8A0053C015E0650D8A0063C025E3E
:100DD80006340E120EA0F4EF06F00D80FFEF06F0B9
:100DE800045000260550D8B0053C01260650D8B05E
:100DF800062802260D900B2EDBEF06F025EF07F0F4
:100E0800D8900036013602360E360450005E055082
:100E1800D8A0053C015E0650D8A0063C025E063408
:100E28000E10010B0D26D8B00C2AD8B4082AD8A465
:100E380025EF07F008320C320D32032AD8B438EF08
:100E480007F00AAE089E0850026E0C50016E0D5055
:100E5800006E40EF07F0010EDCDD40EF07F0020EF8
:100E6800BCEC00F040EF07F0040EB0EC00F040EFEF
:0A0E780007F0080EC3EC00F01200B2
:100E8200800E0601A719006E800E000A005CD8B021
:100E920066D1A7510008016E01C0A7F6800E0118A5
:100EA200006E800E6E0A005CD8A0BAD0640E046E8A
:100EB200A7C600F0C1DC120E0024056E000E00BEB3
:100EC200FF0E066E000E062205C000F006C001F0FD
:100ED200000E06BEFF0E026E036E00360090013653
:100EE20002360336003600900136023603366E0EA5
:100EF2000024F66E940E0120F76E000E0220F86EAA
:100F02000900F5CFA8F60900F5CFA9F60900F5CF3B
:100F1200AAF60900F5CFABF6640E046EA7C600F080
:100F22008BDC08C000F00A0E046E86DC090E002479
:100F3200056E000E00BEFF0E066E000E062205C0F4
:100F420000F006C001F0000E06BEFF0E026E036E38
:100F52000036009001360236033600360090013624
:100F6200023603366E0E0024F66E940E0120F76EE2
:100F7200000E0220F86E0900F5CF00F00900F5CF4F
:100F820001F00900F5CF02F00900F5CF03F0A8C681
:100F920004F0A9C605F0AAC606F0ABC607F0A9DCA4
:100FA20000C0A8F601C0A9F602C0AAF603C0ABF6BB
:100FB2000A0E046EA7C600F03FDC08C000F000C0B5
:100FC20001F0000E00BEFF0E026E036E046E0136CB
:100FD200019002360336043601360190023603369A
:100FE20004366E0E0124F66E940E0220F76E000E89
:100FF2000320F86E0900F5CF00F00900F5CF01F0EB
:101002000900F5CF02F00900F5CF03F0A8C604F0FD
:10101200A9C605F0AAC606F0ABC607F06ADC06D27E
:10102200800E0A0A006E800EA719005C70E20A0E9A
:10103200046EA7C600F000DC090E0024056E000E47
:1010420000BEFF0E066E000E062205C000F006C0AE
:1010520001F0000E06BEFF0E026E036E0036009017
:101062000136023603360036009001360236033668
:101072006E0E0024F66E940E0120F76E000E022012
:10108200F86E0900F5CFA8F60900F5CFA9F6090018
:10109200F5CFAAF60900F5CFABF60A0E046EA7C685
:1010A20000F01DEC04F008C000F000C001F0000EDA
:1010B20000BEFF0E026E036E046E01360190023610
:1010C20003360436013601900236033604366E0EBC
:1010D2000124F66E940E0220F76E000E0320F86EC5
:1010E2000900F5CF00F00900F5CF01F00900F5CFB6
:1010F20002F00900F5CF03F0A8C604F0A9C605F076
:10110200AAC606F0ABC607F07AEC04F08FD1A7C6E8
:1011120000F0000EA7BFFF0E016E026E036E0036D6
:101122000090013602360336003600900136023650
:1011320003366E0E0024F66E940E0120F76E000E3A
:101142000220F86E0900F5CF00F00900F5CF01F09A
:101152000900F5CF02F00900F5CF03F067D1800E48
:10116200A719006E800E6E0A005CD8A0C0D0640E73
:10117200046EA7C600F01DEC04F0120E0024056EEA
:10118200000E00BEFF0E066E000E062205C000F025
:1011920006C001F0000E06BEFF0E026E036E0036A0
:1011A20000900136023603360036009001360236D0
:1011B20003363A0E0024F66E940E0120F76E000EEE
:1011C2000220F86E0900F5CFA8F60900F5CFA9F6BE
:1011D2000900F5CFAAF60900F5CFABF6640E046E4E
:1011E200A7C600F01DEC04F008C000F00A0E046E61
:1011F2001DEC04F0090E0024056E000E00BEFF0E69
:10120200066E000E062205C000F006C001F0000EB8
:1012120006BEFF0E026E036E0036009001360236E5
:101222000336003600900136023603363A0E0024A9
:10123200F66E940E0120F76E000E0220F86E090081
:10124200F5CF00F00900F5CF01F00900F5CF02F06B
:101252000900F5CF03F0A8C604F0A9C605F0AAC696
:1012620006F0ABC607F07AEC04F000C0A8F601C0A5
:10127200A9F602C0AAF603C0ABF60A0E046EA7C610
:1012820000F01DEC04F008C000F000C001F0000EF8
:1012920000BEFF0E026E036E046E0136019002362E
:1012A20003360436013601900236033604363A0E0E
:1012B2000124F66E940E0220F76E000E0320F86EE3
:1012C2000900F5CF00F00900F5CF01F00900F5CFD4
:1012D20002F00900F5CF03F0A8C604F0A9C605F094
:1012E200AAC606F0ABC607F07AEC04F09FD0800ED7
:1012F2000A0A006E800EA719005C71E20A0E046EE3
:10130200A7C600F01DEC04F0090E0024056E000EC5
:1013120000BEFF0E066E000E062205C000F006C0DB
:1013220001F0000E06BEFF0E026E036E0036009044
:101332000136023603360036009001360236033695
:101342003A0E0024F66E940E0120F76E000E022073
:10135200F86E0900F5CFA8F60900F5CFA9F6090045
:10136200F5CFAAF60900F5CFABF60A0E046EA7C6B2
:1013720000F01DEC04F008C000F000C001F0000E07
:1013820000BEFF0E026E036E046E0136019002363D
:1013920003360436013601900236033604363A0E1D
:1013A2000124F66E940E0220F76E000E0320F86EF2
:1013B2000900F5CF00F00900F5CF01F00900F5CFE3
:1013C20002F00900F5CF03F0A8C604F0A9C605F0A3
:1013D200AAC606F0ABC607F07AEC04F027D0A7C67F
:1013E20000F0000EA7BFFF0E016E026E036E003604
:1013F200009001360236033600360090013602367E
:1014020003363A0E0024F66E940E0120F76E000E9B
:101412000220F86E0900F5CF00F00900F5CF01F0C7
:0E1422000900F5CF02F00900F5CF03F012002B
:101430009BC0A9F69CC0AAF69DC0ABF69EC0ACF6B8
:101440000601A76BA86BA851120802E1A7518E08EC
:1014500009E31DEC05F0005201E004D00601A74BA2
:10146000A82BF1D70601120EA85D02E18F0EA75D31
:1014700003E37B0E006E27D0C580C5A023D00001FA
:101480009B519C119D119E111CE00601A951AA11AE
:10149000AB11AC110FE15BC5E1FF5CC5E2FF050ECE
:1014A000E66E59C500F05AC501F011EC05F0010EC9
:1014B000006E09D0010E0601A95F000EAA5BAB5BAE
:0814C000AC5BDBD7006A1200EF
:1014C8009BC0A7F69CC0A8F69DC0A9F69EC0AAF628
:1014D800C582C5A221D000019B519C119D119E116E
:1014E8001AE00601A751A811A911AA110DE15BC5BF
:1014F800E1FF5CC5E2FF060EE66E59C500F05AC56D
:1015080001F011EC05F008D0010E0601A75F000EEE
:0A151800A85BA95BAA5BDDD71200F7
:101522009BC0A9F69CC0AAF69DC0ABF69EC0ACF6C5
:101532009E96C5869EB621D000019B519C119D119D
:101542009E111AE00601A951AA11AB11AC110DE1CD
:101552005BC5E1FF5CC5E2FF030EE66E59C500F014
:101562005AC501F011EC05F008D0010E0601A95F81
:10157200000EAA5BAB5BAC5BDDD70601C9CFA8F658
:10158200A751000A02E1C58A01D0C59A9E96C58874
:101592009BC0A9F69CC0AAF69DC0ABF69EC0ACF655
:1015A2009EB621D000019B519C119D119E111AE003
:1015B2000601A951AA11AB11AC110DE15BC5E1FF06
:1015C2005CC5E2FF030EE66E59C500F05AC501F094
:1015D20011EC05F008D0010E0601A95F000EAA5B0E
:0C15E200AB5BAC5BDDD7A8C600F01200CC
:1015EE009E96A7C6C9FF9BC0A8F69CC0A9F69DC033
:1015FE00AAF69EC0ABF6C7A423D000019B519C1146
:10160E009D119E111CE00601A851A911AA11AB1142
:10161E000FE15BC5E1FF5CC5E2FF040EE66E59C546
:10162E0000F05AC501F011EC05F0010E006E3CD031
:10163E00010E0601A85F000EA95BAA5BAB5BDBD7B0
:10164E009BC0A8F69CC0A9F69DC0AAF69EC0ABF69C
:10165E009EB623D000019B519C119D119E111CE042
:10166E000601A851A911AA11AB110FE15BC5E1FF4B
:10167E005CC5E2FF040EE66E59C500F05AC501F0D6
:10168E0011EC05F0010E006E0FD0010E0601A85FE1
:10169E00000EA95BAA5BAB5BDBD7C5BC02D0006AB0
:0A16AE0003D0C584020E006E120086
:1016B8006E0E0601A75DD8A0CAD0640E046EA7C638
:1016C80000F0D2EC01F0120E0024056E066A000E3E
:1016D800062205C000F006C001F0000E06BEFF0E8F
:1016E800026E036E0036009001360236033600366D
:1016F80000900136023603366E0E0024F66E940E04
:101708000120F76E000E0220F86E0900F5CF00F0F8
:101718000900F5CF01F00900F5CF02F00900F5CF77
:1017280003F0000E046E000E056E000E066E7E0EAF
:10173800076E7AEC04F000C0A8F601C0A9F602C052
:10174800AAF603C0ABF6640E046EA7C600F0D2EC8E
:1017580001F008C000F00A0E046ED2EC01F0090E88
:101768000024056E066A000E062205C000F006C0B9
:1017780001F0000E06BEFF0E026E036E00360090EA
:10178800013602360336003600900136023603363B
:101798006E0E0024F66E940E0120F76E000E0220E5
:1017A800F86E0900F5CF00F00900F5CF01F0090047
:1017B800F5CF02F00900F5CF03F0A8C604F0A9C6DA
:1017C80005F0AAC606F0ABC607F07AEC04F000C034
:1017D800A8F601C0A9F602C0AAF603C0ABF60A0E25
:1017E800046EA7C600F0D2EC01F008C000F000C0FB
:1017F80001F0000E026E036E046E0136019002368F
:1018080003360436013601900236033604366E0E6E
:101818000124F66E940E0220F76E000E0320F86E77
:101828000900F5CF00F00900F5CF01F00900F5CF68
:1018380002F00900F5CF03F0A8C604F0A9C605F028
:10184800AAC606F0ABC607F07AEC04F0B1D0A751EF
:101858000A08D8B07ED00A0E046EA7C600F0D2ECF3
:1018680001F0090E0024056E066A000E062205C066
:1018780000F006C001F0000E06BEFF0E026E036EF9
:1018880000360090013602360336003600900136E5
:10189800023603366E0E0024F66E940E0120F76EA3
:1018A800000E0220F86E0900F5CF00F00900F5CF10
:1018B80001F00900F5CF02F00900F5CF03F0000EA2
:1018C800046E000E056E000E066E7E0E076E7AEC34
:1018D80004F000C0A8F601C0A9F602C0AAF603C029
:1018E800ABF60A0E046EA7C600F0D2EC01F008C0F1
:1018F80000F000C001F0000E026E036E046E0136A7
:10190800019002360336043601360190023603365A
:1019180004366E0E0124F66E940E0220F76E000E49
:101928000320F86E0900F5CF00F00900F5CF01F0AB
:101938000900F5CF02F00900F5CF03F0A8C604F0BE
:10194800A9C605F0AAC606F0ABC607F07AEC04F003
:101958002FD0A7C600F0000E016E026E036E00368F
:101968000090013602360336003600900136023602
:1019780003366E0E0024F66E940E0120F76E000EEC
:101988000220F86E0900F5CF00F00900F5CF01F04C
:101998000900F5CF02F00900F5CF03F0000E046E40
:1019A800000E056E000E066E7E0E076E7AEC04F0D1
:0219B80012001B
:1019BA000B6A0A6A096A086A0E6A0334083604500E
:1019CA00085E0550D8A0053C095E0650D8A0063C22
:1019DA000A5E0750D8A0073C0B5EE86AD8A0010E41
:1019EA000E5E0336070E0C6E0334083609360A36C5
:1019FA000B360E36045003A012D0085E0550D8A04C
:101A0A00053C095E0650D8A0063C0A5E0750D8A0DD
:101A1A00073C0B5EE86AD8A0010E0E5E11D00826BC
:101A2A000550D8B0053C09260650D8B0063C0A260F
:101A3A000750D8B0073C0B26E86AD8B0010E0E262C
:101A4A0003360C2ED1D70234083609360A360B363D
:101A5A000E36045003A012D0085E0550D8A0053CEB
:101A6A00095E0650D8A0063C0A5E0750D8A0073C7B
:101A7A000B5EE86AD8A0010E0E5E11D0082605504A
:101A8A00D8B0053C09260650D8B0063C0A260750AD
:101A9A00D8B0073C0B26E86AD8B0010E0E260236EB
:101AAA00070E0C6E0234083609360A360B360E3625
:101ABA00045002A012D0085E0550D8A0053C095E69
:101ACA000650D8A0063C0A5E0750D8A0073C0B5E19
:101ADA00E86AD8A0010E0E5E11D008260550D8B0CB
:101AEA00053C09260650D8B0063C0A260750D8B04D
:101AFA00073C0B26E86AD8B0010E0E2602360C2ED9
:101B0A00D1D70134083609360A360B360E36045058
:101B1A0002A012D0085E0550D8A0053C095E065006
:101B2A00D8A0063C0A5E0750D8A0073C0B5EE86ABC
:101B3A00D8A0010E0E5E11D008260550D8B0053C7B
:101B4A0009260650D8B0063C0A260750D8B0073CEA
:101B5A000B26E86AD8B0010E0E260136070E0C6E67
:101B6A000134083609360A360B360E36045001A0FF
:101B7A0012D0085E0550D8A0053C095E0650D8A0D0
:101B8A00063C0A5E0750D8A0073C0B5EE86AD8A05C
:101B9A00010E0E5E11D008260550D8B0053C092664
:101BAA000650D8B0063C0A260750D8B0073C0B2688
:101BBA00E86AD8B0010E0E2601360C2ED1D70034B1
:101BCA00083609360A360B360E36045001A012D0F2
:101BDA00085E0550D8A0053C095E0650D8A0063C10
:101BEA000A5E0750D8A0073C0B5EE86AD8A0010E2F
:101BFA000E5E11D008260550D8B0053C09260650BD
:101C0A00D8B0063C0A260750D8B0073C0B26E86A2B
:101C1A00D8B0010E0E260036070E0C6E00340836B8
:101C2A0009360A360B360E36045000A012D0085E6A
:101C3A000550D8A0053C095E0650D8A0063C0A5EAD
:101C4A000750D8A0073C0B5EE86AD8A0010E0E5ECA
:101C5A0011D008260550D8B0053C09260650D8B040
:101C6A00063C0A260750D8B0073C0B26E86AD8B0CB
:101C7A00010E0E2600360C2ED1D700B00ED004501D
:101C8A0008260550D8B0053C09260650D8B0063CAF
:0C1C9A000A260750D8B0073C0B261200A9
:041CA600C5841200DF
:101CAA000A6A0350D8A40A800750D8A40A820A50A4
:101CBA00D8B4B8EF0EF0030AD8B471EF0EF00AB038
:101CCA006CEF0EF006AEB6EF0EF0B4EF0EF002AE09
:101CDA00B4EF0EF0B6EF0EF00250800B0A6E029EC1
:101CEA000650800B069E0A18D8B482EF0EF00A50EE
:101CFA00D8B4B4EF0EF0B6EF0EF00750035CD8B4C8
:101D0A008CEF0EF0D8A0A8EF0EF0AEEF0EF0065052
:101D1A00025CD8B496EF0EF0D8A0A8EF0EF0AEEFA2
:101D2A000EF00550015CD8B4A0EF0EF0D8A0A8EFD1
:101D3A000EF0AEEF0EF00450005CD8B4B8EF0EF01F
:101D4A00D8B0AEEF0EF00A52D8B4B6EF0EF0B4EF38
:101D5A000EF00A52D8B4B4EF0EF0B6EF0EF0D880F7
:0E1D6A001200D8901200D880D8841200120007
:101D78000B6A0C6A086A0350D8B440EF0FF002C02F
:101D88000AF0028E9E0E035E03AE30EF0FF0036C76
:101D9800080E035CD8A0FDEF0EF0036E083600C0F5
:101DA80008F001C000F002C001F0026A080E035CEE
:101DB800D8A0FDEF0EF0036E083600C008F001C091
:101DC80000F0016A080E035CD8A0FDEF0EF0036E68
:101DD800083600C008F0006A080E035CD8A0FDEFC2
:101DE8000EF0036E0836086A0350D8A4D89009EF9D
:101DF8000FF00350D8B409EF0FF0D8900232013237
:101E080000320832032E01EF0FF00BBC08A01AEFC6
:101E18000FF0D8A01AEF0FF0082AD8B4002AD8B4C7
:101E2800012AD8B4022A02BE44EF0FF00AAE40EFEE
:101E38000FF0021E011E001E081E082AD8B4002A30
:101E4800D8B4012AD8B4022A40EF0FF0026A016A16
:101E5800006A086A40EF0FF00B800BAE4BEF0FF0F3
:101E6800026A0AAE4BEF0FF0026E016E006E086E4A
:101E78000A3602324BEF0FF00C6A000E4CEF0FF0EF
:101E8800010E0C6E000E6CEC04F04CEF0FF0FF0E20
:101E98000250036E0150026E0050016E0850006E31
:021EA800120026
:101EAA000B1E0A1E091E081E082AD8B4092AD8B40D
:081EBA000A2AD8B40B2A120019
:101EC2000450085E0550D8A0053C095E0650D8A013
:101ED200063C0A5E0750D8A0073C0B5E0336070E8D
:101EE2000C6E0334083609360A360B36045003A04A
:101EF2000ED0085E0550D8A0053C095E0650D8A059
:101F0200063C0A5E0750D8A0073C0B5E0DD008269F
:101F12000550D8B0053C09260650D8B0063C0A2622
:101F22000750D8B0073C0B2603360C2EDAD7023402
:101F3200083609360A360B36045003A00ED0085E66
:101F42000550D8A0053C095E0650D8A0063C0A5EA2
:101F52000750D8A0073C0B5E0DD008260550D8B01C
:101F6200053C09260650D8B0063C0A260750D8B0D0
:101F7200073C0B260236070E0C6E02340836093671
:101F82000A360B36045002A00ED0085E0550D8A0C7
:101F9200053C095E0650D8A0063C0A5E0750D8A050
:101FA200073C0B5E0DD008260550D8B0053C09262B
:101FB2000650D8B0063C0A260750D8B0073C0B267C
:101FC20002360C2EDAD70134083609360A360B36B9
:101FD200045002A00ED0085E0550D8A0053C095E50
:101FE2000650D8A0063C0A5E0750D8A0073C0B5EFC
:101FF2000DD008260550D8B0053C09260650D8B0A9
:10200200063C0A260750D8B0073C0B260136070EBD
:102012000C6E0134083609360A360B36045001A01C
:102022000ED0085E0550D8A0053C095E0650D8A027
:10203200063C0A5E0750D8A0073C0B5E0DD008266E
:102042000550D8B0053C09260650D8B0063C0A26F1
:102052000750D8B0073C0B2601360C2EDAD70034D5
:10206200083609360A360B36045001A00ED0085E37
:102072000550D8A0053C095E0650D8A0063C0A5E71
:102082000750D8A0073C0B5E0DD008260550D8B0EB
:10209200053C09260650D8B0063C0A260750D8B09F
:1020A200073C0B260036070E0C6E00340836093644
:1020B2000A360B36045000A00ED0085E0550D8A098
:1020C200053C095E0650D8A0063C0A5E0750D8A01F
:1020D200073C0B5E0DD008260550D8B0053C0926FA
:1020E2000650D8B0063C0A260750D8B0073C0B264B
:1020F20000360C2EDAD700B00ED004500826055058
:10210200D8B0053C09260650D8B0063C0A2607502E
:08211200D8B0073C0B261200B7
:10211A000601A751390806E3300EA75D03E3010E55
:08212A00006E01D0006A1200F2
:102132000B6A0A6A096A00500402F4CF09F0F3CF6D
:1021420008F001500502F4CF0BF0F3CF0AF0005073
:102152000502F3500926F4500A22E86A0B220150C4
:102162000402F3500926F4500A22E86A0B2208C03E
:1021720000F009C001F00AC002F00BC003F0120027
:10218200086A096A100E0C6E0134083609360450CA
:10219200085E0550D8A0053C095ED8B007D00450AF
:1021A20008260550D8B0053C0926D89000360136DD
:0621B2000C2EEAD712001A
:1021B8000601806B7F5109081DE20A0E046E7FC676
:1021C80000F0D2EC01F000C080F600C080F6803745
:1021D80080918037809180378091803780910A0E76
:1021E800046E7FC600F0D2EC01F008C000F0005089
:0E21F800801302D07FC680F680C600F0120071
:1022060018EC0AF0D00E0601A76FF7EC0AF07FC6AD
:10221600A7F6F7EC0AF080C6A7F6F7EC0AF040DD61
:022226001200A4
:102228008B921A0E0D6E0D2EFED7000081A429D0B8
:102238007FC6A7F656EC06F088C6A7F656EC06F059
:10224800000000007FC6A7F656EC06F089C6A7F680
:1022580056EC06F0000000007FC6A7F656EC06F024
:102268008AC6A7F656EC06F0000000007FC6A7F65F
:1022780056EC06F08BC6A7F656EC06F000000000F8
:1022880078D07FC6A7F656EC06F08BC6A7F656ECB4
:1022980006F0000000007FC6A7F656EC06F08AC6D6
:1022A800A7F656EC06F0000000007FC6A7F656EC2D
:1022B80006F089C6A7F656EC06F0000000007FC6B7
:1022C800A7F656EC06F088C6A7F656EC06F000000E
:1022D80000007FC6A7F656EC06F087C6A7F656ECB0
:1022E80006F0000000007FC6A7F656EC06F086C68A
:1022F800A7F656EC06F0000000007FC6A7F656ECDD
:1023080006F085C6A7F656EC06F0000000007FC66A
:10231800A7F656EC06F084C6A7F656EC06F00000C1
:1023280000007FC6A7F656EC06F083C6A7F656EC63
:1023380006F0000000007FC6A7F656EC06F082C63D
:10234800A7F656EC06F0000000007FC6A7F656EC8C
:1023580006F081C6A7F656EC06F0000000007FC61E
:10236800A7F656EC06F080C6A7F656EC06F0000075
:1023780000001A0E0D6E0D2EFED700008B82120083
:102388007FC602F080C603F002C000F003C001F06F
:10239800024A032A00C0E9FF01C0EAFFEE5201E049
:1023A800F3D706017F51025C006E80510358016E1D
:0A23B800010E005E000E015A120033
:1023C2007FC6E9FF80C6EAFFEE520CE07FC6E9FF56
:1023D20080C6EAFFEECFADF6DAEC00F006017F4BE5
:1023E200802BEED71A0E0D6E0D2EFED700001200B6
:1023F2007FC600F00032009E0032009E0032009E36
:102402000032009E80C6E1FF81C6E2FF300E00244A
:10241200E66E010E06018025E16E000E8121E26E5C
:102422000F0E7F15006E300E002600C0E6FF020E72
:0E2432008025E16E000E8121E26EE66A120046
:10244000000EF2BE010E0601806FF29E18EC0AF03B
:10245000D00E0601A76FF7EC0AF07FC6A7F6F7ECDF
:102460000AF064EC0AF0D10E0601A76FF7EC0AF04F
:102470000601A76B91EC0AF000C081F614DC06019E
:0E2480008051010AD8B4F28E81C600F012001D
:10248E000450000A12E10550000A0FE10650000A3E
:10249E000CE10750000A09E1FF0E006EFF0E016EFF
:1024AE00FF0E026E7F0E036E97D00C6A07BE0C2ACB
:1024BE000D6A0B6A0A6A096A086A03500210011053
:1024CE000010D8B484D0035007180E6E0EBE0D1E29
:1024DE0007AE0BD0041E051E061E071E042AD8B416
:1024EE00052AD8B4062AD8B4072A03AE0BD0001E8C
:1024FE00011E021E031E002AD8B4012AD8B4022AD5
:10250E00D8B4032A035007100E6E0EBE1CD0D2DCB8
:10251E000CBE36D00DAE5BD0001E011E021E031E79
:10252E00002AD8B4012AD8B4022AD8B4032A081E25
:10253E00091E0A1E0B1E082AD8B4092AD8B40A2A64
:10254E00D8B40B2A44D007AE15D003BE0DD003501D
:10255E000B6E02500A6E0150096E0050086E036A2F
:10256E00026A016A006AD6D7036A026A016A006AC1
:10257E00002A000C031E021E011E001E0C8EC7D761
:10258E00082AD8B4092AD8B40A2AD8B40B2A045077
:10259E00085CD8A4BFD70550095CD8A4BBD7065099
:1025AE000A5CD8A4B7D707500B5CD8A4B3D70B6A74
:1025BE000A6A096A086A002AD8B4012AD8B4022A1B
:1025CE00D8B4032A03AEA6D70E6A0E88FF0C0E6A85
:0A25DE000CA001D063DC000F120016
:1025E8007FC604F080C605F006018351841124E0FB
:1025F800010E835F000E845B04C002F005C003F087
:10260800044A052A81C600F082C601F0814B822B5C
:1026180000C0E9FF01C0EAFF02C0E1FF03C0E2FF1A
:10262800EECFE6FF02C0E9FF03C0EAFFEECF00F0FD
:10263800005201E101D0D8D783C600F084C601F06A
:10264800010E835F000E845B0050011008E004C097
:10265800E1FF05C0E2FFE66A044A052AEDD77FC616
:0826680000F080C601F0120031
:102670007FC604F080C605F004C002F005C003F078
:10268000044A052A81C600F082C601F00601814B8A
:10269000822B00C0E9FF01C0EAFF02C0E1FF03C0D6
:1026A000E2FFEECFE6FF02C0E9FF03C0EAFFEE5211
:0E26B00001E0E2D77FC600F080C601F0120004
:1026BE000601836B050E835D0AE283518125E16E6F
:1026CE00000E8221E26E200EE66E832BF3D783512D
:1026DE008125E16E000E8221E26EE66A8307835148
:1026EE008125846F000E8221856F0A0E046E000E06
:1026FE00056E7FC600F080C601F03CDD08C000F01C
:10270E0009C001F0300E002684C6E1FF85C6E2FF47
:10271E0000C0E6FF0A0E046E000E056E7FC600F0C6
:10272E0080C601F027DD00C07FF601C080F6000EE6
:10273E00011802E1000E001801E102D08307CFD785
:02274E00120077
:102750000C6A0E6A0250D8A4C1EF13F001C002F057
:1027600000C001F0006A0E860250D8A4C1EF13F039
:1027700001C002F0016A0E960E880250D8B4D3EF61
:1027800013F00E50035ED8A4D8A0D9EF13F0D89060
:1027900002BEDFEF13F0003601360236032EC8EF1B
:1027A00013F0D9EF13F0010E0C6EBCEC00F0E3EF68
:1027B00013F0020E0C6EC3EC00F0E3EF13F0040E06
:0827C0000C6ED0EC00F01200D9
:1027C800A69C80C6AAFF7FC6A9FFA69EA680A8CF02
:0427D80000F01200FB
:1027DC000D0E0601AD6FDAEC00F00A0E0601AD6FBE
:0627EC00DAEC00F012001F
:1027F2007FC6E9FF80C6EAFFEECF81F6000E060132
:10280200826F000E826F000E821902E1200E811982
:1028120007E0000E821902E1090E811901E003D0DE
:102822007F4B802BE5D7836B846B856B866B000EA9
:10283200821902E12D0E811905E1854B862B7F4B12
:10284200802B08D0000E821902E12B0E811902E1C1
:102852007F4B802B7FC6E9FF80C6EAFFEECF81F671
:10286200000E826F000E826F81C6A7F655DC005201
:1028720018E083C600F084C601F00A0E046E000E52
:10288200056E56DC300E815D026E000E8259036EBB
:1028920002500024836F03500120846F7F4B802BF2
:1028A200D9D78551861108E083510008006E84C68D
:1028B20001F0000E015604D083C600F084C601F078
:0228C200120002
:1028C4000601826B7FC6E9FF80C6EAFFEECF81F680
:1028D4008151000A0FE081C6ADF6DAEC00F0060182
:1028E400822B82517F25E96E000E8021EA6EEECFA5
:0628F40081F6EED7120090
:1028FA00220E0C6E086A096A0A6A0B6A0C06D8B4B8
:10290A001FD0D8900B320A3209320832033202320F
:10291A0001320032D8A0F2D70C06D8B409D004503C
:10292A0008260550092206500A2207500B22EAD728
:10293A00045008260550092206500A2207500B2285
:02294A00120079
:10294C0081C6F6FF82C6F7FF83C6F8FF0900F5CFF4
:10295C0000F0005218E081C6F6FF82C6F7FF83C66E
:10296C00F8FF0900F5CF00F07FC6E1FF80C6E2FF5B
:10297C0000C0E6FF06017F4B802B010E8127000E65
:10298C0082238323DDD77FC6E1FF80C6E2FFE66AA0
:02299C00120027
:10299E0006019F6BA06B936B946B81C600F082C691
:1029AE0001F083C602F0010E8127000E82238323DD
:1029BE0000C0F6FF01C0F7FF02C0F8FF0900F5CF17
:1029CE0000F000C090F60052D8B4DDEF24F0905124
:1029DE00250A0BE07FC6E1FF80C6E2FF90C6E6FF48
:1029EE007F4B802B9F4BA02BD8D7916B926B936B09
:1029FE00946B23D09387010E8127000E82238323AD
:102A0E0059D09381010E8127000E8223832352D049
:102A1E009383010E8127000E822383234BD094874C
:102A2E00010E8127000E8223832344D09385010E4D
:102A3E008127000E822383233DD081C6F6FF82C6F6
:102A4E00F7FF83C6F8FF0900F5CF01F001502D0AFC
:102A5E00D1E081C6F6FF82C6F7FF83C6F8FF0900F4
:102A6E00F5CF01F00150200ACCE081C6F6FF82C6F8
:102A7E00F7FF83C6F8FF0900F5CF01F001502B0ACE
:102A8E00C7E081C6F6FF82C6F7FF83C6F8FF0900CE
:102A9E00F5CF01F00150230AC2E081C6F6FF82C6CF
:102AAE00F7FF83C6F8FF0900F5CF01F00150300A99
:102ABE00BDE001D09ED793A301D0939193A701D0EF
:102ACE00939581C6F6FF82C6F7FF83C6F8FF09000D
:102ADE00F5CF00F0000E016E00C0A7F68DEC10F0E1
:102AEE00005236E0916B926B91C600F092C601F0E7
:102AFE000A0E046E000E056E99EC10F081C6F6FFFC
:102B0E0082C6F7FF83C6F8FF0900F5CF02F0025028
:102B1E000024916F000E0120926F300E915F000E17
:102B2E00925B010E8127000E8223832381C6F6FF5E
:102B3E0082C6F7FF83C6F8FF0900F5CF00F0000E3E
:102B4E00016E00C0A7F68DEC10F00052CDE133D02F
:102B5E0081C6F6FF82C6F7FF83C6F8FF0900F5CFE0
:102B6E0001F001502A0A27E184C6E9FF85C6EAFF73
:102B7E00EECF00F0EECF01F000C0E9FF01C0EAFF9A
:102B8E00EECF91F6EECF92F684C6E9FF85C6EAFF48
:102B9E00020EEE24006E000EEE20016E84C6E1FFE2
:102BAE0085C6E2FF00C0E6FF01C0E6FF010E8127E9
:102BBE00000E8223832381C6F6FF82C6F7FF83C6EB
:102BCE00F8FF0900F5CF01F001502E0A70E1010E59
:102BDE008127000E8223832381C6F6FF82C6F7FF6C
:102BEE0083C6F8FF0900F5CF01F001502A0A28E14B
:102BFE0084C6E9FF85C6EAFFEECF00F0EECF01F006
:102C0E0000C0E9FF01C0EAFFEECF8EF6EECF8FF6E1
:102C1E0084C6E9FF85C6EAFF020EEE24006E000EA2
:102C2E00EE20016E84C6E1FF85C6E2FF00C0E6FF1E
:102C3E0001C0E6FF010E8127000E8223832336D0CA
:102C4E008E6B8F6B81C6F6FF82C6F7FF83C6F8FFC9
:102C5E000900F5CF00F0000E016E00C0A7F68DEC56
:102C6E0010F0005223E08EC600F08FC601F00A0E5F
:102C7E00046E000E056E99EC10F081C6F6FF82C64A
:102C8E00F7FF83C6F8FF0900F5CF02F002500024CB
:102C9E008E6F000E01208F6F300E8E5F000E8F5BD9
:102CAE00010E8127000E82238323CCD703D08E6B97
:102CBE008F6B948981C600F082C601F083C602F044
:102CCE00010E8127000E8223832300C0F6FF01C070
:102CDE00F7FF02C0F8FF0900F5CF90F6F9D09FC6B6
:102CEE0000F0A0C601F0E1EF24F09389E3D79485BC
:102CFE002ED1938B94812BD1948329D1938D27D16F
:102D0E0026D1938B938F23D184C6E9FF85C6EAFF24
:102D1E00EECF00F0EECF01F000C0E9FF01C0EAFFF8
:102D2E00EECF9BF6EECF9CF684C6E9FF85C6EAFF92
:102D3E00020EEE24006E000EEE20016E84C6E1FF40
:102D4E0085C6E2FF00C0E6FF01C0E6FF000E9C193B
:102D5E0002E1000E9B1904E19F0E9B6F000E9C6F0B
:102D6E009D6B9E6B9D519B25E96E9E519C21EA6E3B
:102D7E00EE520BE0010E9D25006E000E9E21016E9F
:102D8E0000C09DF601C09EF6EDD78E518F110AE060
:102D9E009E518F5D02E19D518E5D04E28EC69DF6C1
:102DAE008FC69EF692519E5D02E191519D5D05E2A8
:102DBE009D51915F9E51925B02D0916B926B93B736
:102DCE0016D091C600F092C601F0010E915F000E72
:102DDE00925B005001100BE07FC6E1FF80C6E2FF60
:102DEE00200EE66E7F4B802B9F4BA02BEAD79DC605
:102DFE0002F09EC603F0010E9D5D006E000E9E5900
:102E0E00016E00C09DF601C09EF60250031019E03F
:102E1E009BC6E9FF9CC6EAFF7FC6E1FF80C6E2FFC4
:102E2E00EECFE6FF7F4B802B010E9B25006E000E32
:102E3E009C21016E00C09BF601C09CF69F4BA02BFF
:102E4E00D6D793A716D091C600F092C601F0010E08
:102E5E00915F000E925B005001100BE07FC6E1FF08
:102E6E0080C6E2FF200EE66E7F4B802B9F4BA02B81
:102E7E00EAD793D584C6E9FF85C6EAFFEECF00F008
:102E8E00EECF01F000C0E9FF01C0EAFFEECF90F6F1
:102E9E0084C6E9FF85C6EAFF020EEE24006E000E20
:102EAE00EE20016E84C6E1FF85C6E2FF00C0E6FF9C
:102EBE0001C0E6FF900E9B6F060E9C6F010E9D6F7C
:102ECE00000E9E6F62D7C00E9313000E94133FD068
:102EDE009051000AD8B403D790516C0AD8B405D7D4
:102EEE0090514C0AD8B401D79051660AD8B4FFD687
:102EFE009051450AD8B4FDD69051650AD8B4FAD689
:102F0E009051670AD8B4F8D690516F0AD8B4F6D655
:102F1E009051640AD8B4F4D69051690AD8B4F0D658
:102F2E009051700AD8B4EDD69051580AD8B4E9D65B
:102F3E009051780AD8B4E6D69051730AD8B4E4D634
:102F4E009051630A97E09051750ABDE0B3D7000E19
:102F5E009315006E9451070B016E00500110D8B4FA
:102F6E0084EF20F094A904D0060E8E6F000E8F6FA2
:102F7E0084C6E9FF85C6EAFFEECF00F0EECF01F082
:102F8E0000C0E9FF01C0EAFFEECF95F6EECF96F650
:102F9E00EECF97F6EECF98F684C6E9FF85C6EAFF28
:102FAE00040EEE24006E000EEE20016E84C6E1FFCC
:102FBE0085C6E2FF00C0E6FF01C0E6FF046A056AAF
:102FCE00066A076A95C600F096C601F097C602F02B
:102FDE0098C603F055EC0EF0010ED8B0000E006E40
:102FEE00005205E0977F030E9313000E9413996B16
:102FFE009A6B95C600F096C601F097C602F098C679
:10300E0003F0046A056A066A076A2AEC05F0000EE8
:10301E00D8A4010E006E0052D8B48AD098C600F023
:10302E00016A026A036AFF0E0016000E01167E0E7A
:10303E00005E000E015A00C099F601C09AF6010E0C
:10304E00005E000E015A00C099F601C09AF6030EFA
:10305E00046E000E056E99EC10F000C099F601C0DA
:10306E009AF60A0E046E000E056E41EC05F000C0D5
:10307E0099F601C09AF6800E0118026E800E025C5F
:10308E0002E1000E005C05E2010E0601995F000EE2
:10309E009A5B060199510008A76F41EC07F095C69F
:1030AE0004F096C605F097C606F098C607F07AECBF
:1030BE0004F000C09BF601C09CF602C09DF603C052
:1030CE009EF6000E046E000E056E000E066E7F0E4E
:1030DE00076E9BC600F09CC601F09DC602F09EC610
:1030EE0003F055EC0EF0010ED8B0000E006E00523B
:1030FE0005E0010E995F000E9A5B1AD0000E046E69
:10310E00000E056E200E066E820E076E9BC600F038
:10311E009CC601F09DC602F09EC603F055EC0EF063
:10312E00000ED8B0010E006E005202E0994B9A2BA1
:10313E00800E006E800E9A19005C02E19951000813
:10314E0003E3010E906F02D099C690F694B118D099
:10315E0094A315D0800E9A19006E7F0E005C02E1CA
:10316E00FC0E995D0BE3800E9A19006E800E8F197E
:10317E00005C02E18E51995D01E201D001D0EFD3E6
:10318E008E518F1106E094A304D0010E8E5F000EB7
:10319E008F5B8F51000802E18E51080803E2080E82
:1031AE00906F02D08EC690F695C600F096C601F0CE
:1031BE0097C602F098C603F0046A056A066A076AA3
:1031CE002AEC05F0000ED8A4010E006E0052D8B401
:1031DE004BD199C6A7F641EC07F000C004F001C030
:1031EE0005F002C006F003C007F095C600F096C6C3
:1031FE0001F097C602F098C603F084EC06F000C00A
:10320E0095F601C096F602C097F603C098F6060131
:10321E0090510008A76F41EC07F000C004F001C008
:10322E0005F002C006F003C007F095C600F096C682
:10323E0001F097C602F098C603F084EC06F000C0C9
:10324E00A1F601C0A2F602C0A3F603C0A4F6A1C661
:10325E0095F6A2C696F6A3C697F6A4C698F6A1C68C
:10326E0000F0A2C601F0A3C602F0A4C603F0A4ECBF
:10327E0005F03FEC06F000C004F001C005F002C0FE
:10328E0006F003C007F0A1C600F0A2C601F0A3C667
:10329E0002F0A4C603F052EC06F0000E046E000E0F
:1032AE00056E000E066E7E0E076E55EC0EF0000ECD
:1032BE00D8B0010E006E00521AE095C600F096C608
:1032CE0001F097C602F098C603F0000E046E000ED1
:1032DE00056E000E066E7E0E076EE1EC01F000C06C
:1032EE0095F601C096F602C097F603C098F695C6FD
:1032FE0000F096C601F097C602F098C603F0A4EC53
:10330E0005F006019051010F096E0A6A000E0A229D
:10331E0009C004F00AC005F0000E0ABEFF0E066ECC
:10332E00076E0436049005360636073604360490CA
:10333E00053606360736080E0424F66E960E052060
:10334E00F76E000E0620F86E0900F5CF05F00900A5
:10335E00F5CF06F00900F5CF07F00900F5CF08F01C
:10336E000850035C08E10750025C05E10650015C61
:10337E0002E10550005C1EE3060195C600F096C6FC
:10338E0001F097C602F098C603F0CD0E046ECC0E77
:10339E00056E4C0E066E7B0E076E7AEC04F000C0C6
:1033AE0095F601C096F602C097F603C098F6994BB3
:1033BE009A2B5AD095C600F096C601F097C602F029
:1033CE0098C603F0A4EC05F090C604F0000E056E4E
:1033DE00066E076E0436049005360636073604363A
:1033EE000490053606360736080E0424F66E960E41
:1033FE000520F76E000E0620F86E0900F5CF05F0D9
:10340E000900F5CF06F00900F5CF07F00900F5CF5A
:10341E0008F00850035C08E10750025C05E1065015
:10342E00015C02E10550005C1FE2060195C600F04A
:10343E0096C601F097C602F098C603F0000E046E11
:10344E00000E056E200E066E820E076E7AEC04F0EC
:10345E0000C095F601C096F602C097F603C098F626
:10346E00010E995F000E9A5B060194A393D094B758
:10347E0091D0800E000A006E800E8F19005C02E162
:10348E008E510A0804E20A0E8E6F000E8F6F95C6DB
:10349E0000F096C601F097C602F098C603F0A4ECB1
:1034AE0005F000C09BF601C09CF602C09DF603C05D
:1034BE009EF69B519C119D119E1142E00A0E046EC8
:1034CE00000E056E066E076E9BC600F09CC601F0E0
:1034DE009DC602F09EC603F0DDEC0CF008C000F0B5
:1034EE0009C001F00AC002F00BC003F0000E046E1A
:1034FE00031808E10450021805E10450011802E116
:10350E000050000A1DE1010E8E5F000E8F5B0A0E49
:10351E00046E000E056E066E076E9BC600F09CC60E
:10352E0001F09DC602F09EC603F0DDEC0CF000C06B
:10353E009BF601C09CF602C09DF603C09EF6B9D75D
:10354E00800E8F19006E800E005C02E190518E5D30
:10355E0021E28E51905DA76F41EC07F000C004F0A0
:10356E0001C005F002C006F003C007F095C600F0DA
:10357E0096C601F097C602F098C603F084EC06F0EA
:10358E0000C095F601C096F602C097F603C098F6F5
:10359E008EC690F6050E06018E25006E000E8F214A
:1035AE00016E0050915F0150925B8E518F1103E1BD
:1035BE0094B701D004D0010E915F000E925B030E02
:1035CE009315006E94C601F0000E01160050011006
:1035DE0004E0010E915F000E925B93A539D093A388
:1035EE0012D093A103D02D0E866F02D02B0E866FB4
:1035FE007FC6E1FF80C6E2FF86C6E6FF7F4B802BCB
:10360E009F4BA02B0CD093A10AD07FC6E1FF80C6A2
:10361E00E2FF200EE66E7F4B802B9F4BA02B800E81
:10362E00006E800E9219005C02E1915100080FE2CB
:10363E007FC6E1FF80C6E2FF300EE66E7F4B802B29
:10364E009F4BA02B010E915F000E925BE8D73AD0F4
:10365E0093B718D0800E006E800E9219005C02E1B6
:10366E00915100080FE27FC6E1FF80C6E2FF200EF7
:10367E00E66E7F4B802B9F4BA02B010E915F000EB1
:10368E00925BE8D793A312D093A103D02D0E876F30
:10369E0002D02B0E876F7FC6E1FF80C6E2FF87C682
:1036AE00E6FF7F4B802B9F4BA02B0CD093A10AD013
:1036BE007FC6E1FF80C6E2FF200EE66E7F4B802BB9
:1036CE009F4BA02B95C600F096C601F097C602F050
:1036DE0098C603F0A4EC05F000C09BF601C09CF662
:1036EE0002C09DF603C09EF690C600F0000E016E5D
:1036FE00026E036E00360090013602360336003637
:10370E000090013602360336080E0024F66E960E31
:10371E000120F76E000E0220F86E0900F5CF04F0BE
:10372E000900F5CF05F00900F5CF06F00900F5CF39
:10373E0007F09BC600F09CC601F09DC602F09EC627
:10374E0003F0DDEC0CF0300E00267FC6E1FF80C6E4
:10375E00E2FF00C0E6FF7F4B802B9F4BA02B8E51CC
:10376E008F1103E194B701D06FD07FC6E1FF80C601
:10377E00E2FF2E0EE66E7F4B802B9F4BA02B9051BF
:10378E008E5F000E8F5B90534DE0900790C600F059
:10379E00000E016E026E036E003600900136023688
:1037AE00033600360090013602360336080E00242A
:1037BE00F66E960E0120F76E000E0220F86E0900CE
:1037CE00F5CF04F00900F5CF05F00900F5CF06F0AE
:1037DE000900F5CF07F09BC600F09CC601F09DC610
:1037EE0002F09EC603F0DDEC0CF00A0E046E000E25
:1037FE00056E066E076EDDEC0CF008C000F009C019
:10380E0001F00AC002F00BC003F0300E00267FC696
:10381E00E1FF80C6E2FF00C0E6FF7F4B802B9F4B8F
:10382E00A02BB1D78E518F110FE07FC6E1FF80C65E
:10383E00E2FF300EE66E7F4B802B9F4BA02B010ECE
:10384E008E5F000E8F5BEED793AB0BD07FC6E1FF82
:10385E0080C6E2FF450EE66E7F4B802B9F4BA02B62
:10386E000AD07FC6E1FF80C6E2FF650EE66E7F4B93
:10387E00802B9F4BA02B800E9A19006E800E005C41
:10388E0002E1000E995D11E299510008996F9A516B
:10389E00000E9A577FC6E1FF80C6E2FF2D0EE66E40
:1038AE007F4B802B9F4BA02B0AD07FC6E1FF80C69B
:1038BE00E2FF2B0EE66E7F4B802B9F4BA02B0A0E4A
:1038CE00046E000E056E99C600F09AC601F041EC2A
:1038DE0005F0300E00267FC6E1FF80C6E2FF00C075
:1038EE00E6FF06017F4B802B9F4BA02B0A0E046E2A
:1038FE00000E056E99C600F09AC601F041EC05F077
:10390E0008C000F009C001F0300E00267FC6E1FFAE
:10391E0080C6E2FF00C0E6FF06017F4B802B9F4B67
:10392E00A02B93A71AD0800E006E800E9219005C09
:10393E0002E19151000811E27FC6E1FF80C6E2FF6D
:10394E00200EE66E7F4B802B9F4BA02B010E915FBE
:10395E00000E925B91519211EFE1D4EF14F094A30B
:10396E00F3D0800E9A19006E800E005C02E1000EFC
:10397E00995D0AE2010E995D006E000E9A59016E74
:10398E0000508E5F01508F5B95C600F096C601F019
:10399E0097C602F098C603F0A4EC05F000C09BF6A3
:1039AE0001C09CF602C09DF603C09EF6010E906FFC
:1039BE0090510A0A34E090C600F0000E016E026EBD
:1039CE00036E003600900136023603360036009044
:1039DE00013602360336080E0024F66E960E0120CE
:1039EE00F76E000E0220F86E0900F5CF01F0090007
:1039FE00F5CF02F00900F5CF03F00900F5CF04F082
:103A0E0004509E5D08E103509D5D05E102509C5DF2
:103A1E0002E101509B5D01E202D0902BC9D790517B
:103A2E008E5DA56F000E8F59A66FA5C68EF6A6C623
:103A3E008FF69BC600F09CC601F09DC602F09EC696
:103A4E0003F03FEC06F000C004F001C005F002C028
:103A5E0006F003C007F095C600F096C601F097C6B3
:103A6E0002F098C603F052EC06F000C0A1F601C0B9
:103A7E00A2F602C0A3F603C0A4F6A5C6A7F641ECB3
:103A8E0007F0A1C604F0A2C605F0A3C606F0A4C6B0
:103A9E0007F07AEC04F0000E046E000E056E000EB8
:103AAE00066E7E0E076EE1EC01F0A4EC05F000C090
:103ABE009BF601C09CF602C09DF603C09EF68E5189
:103ACE008F1142E00A0E046E000E056E066E076E32
:103ADE009BC600F09CC601F09DC602F09EC603F088
:103AEE00DDEC0CF008C000F009C001F00AC002F0D5
:103AFE000BC003F0000E046E031808E10450021808
:103B0E0005E10450011802E10050000A1DE10A0E01
:103B1E00046E000E056E066E076E9BC600F09CC608
:103B2E0001F09DC602F09EC603F0DDEC0CF000C065
:103B3E009BF601C09CF602C09DF603C09EF6010ED8
:103B4E008E5F000E8F5BBBD7800E006E800E8F19BE
:103B5E00005C02E18E510C0816E38EC6A7F65CECF3
:103B6E000BF095C604F096C605F097C606F098C6FB
:103B7E0007F0E1EC01F000C095F601C096F602C028
:103B8E0097F603C098F695C600F096C601F097C654
:103B9E0002F098C603F0046A056A066A076A2AEC00
:103BAE0005F0000ED8A4010E006E0052D8B477D0E6
:103BBE0095C600F096C601F097C602F098C603F0BF
:103BCE00A4EC05F0000E046E031808E10450021870
:103BDE0005E10450011802E10050000A60E1800E78
:103BEE00006E800E9A19005C02E19951010857E2AD
:103BFE0099C6A7F641EC07F000C004F001C005F02D
:103C0E0002C006F003C007F095C600F096C601F09C
:103C1E0097C602F098C603F084EC06F05F0E046EB1
:103C2E00700E056E090E066E810E076E55EC0EF0C7
:103C3E00010ED8B0000E006E005206E0090E06010D
:103C4E00995F000E9A5B05D00601080E995F000E73
:103C5E009A5B99C6A7F641EC07F000C004F001C0CC
:103C6E0005F002C006F003C007F095C600F096C638
:103C7E0001F097C602F098C603F084EC06F0A4ECAF
:103C8E0005F000C09BF601C09CF602C09DF603C075
:103C9E009EF60601956B966B976B986B38D095C612
:103CAE0000F096C601F097C602F098C603F0A4EC99
:103CBE0005F000C09BF601C09CF602C09DF603C045
:103CCE009EF69BC600F09CC601F09DC602F09EC6F5
:103CDE0003F03FEC06F000C004F001C005F002C096
:103CEE0006F003C007F095C600F096C601F097C621
:103CFE0002F098C603F052EC06F000C095F601C033
:103D0E0096F602C097F603C098F6996B9A6B010E61
:103D1E00906F90510A0A34E090C600F0000E016ECA
:103D2E00026E036E00360090013602360336003600
:103D3E000090013602360336080E0024F66E960EFB
:103D4E000120F76E000E0220F86E0900F5CF01F08B
:103D5E000900F5CF02F00900F5CF03F00900F5CF09
:103D6E0004F004509E5D08E103509D5D05E1025094
:103D7E009C5D02E101509B5D01E202D0902BC9D700
:103D8E0090518E25006E000E8F21016E99510026E6
:103D9E009A5101220050915F0150925B94B704D06A
:103DAE008E518F1101E104D0010E915F000E925BD6
:103DBE00030E9315006E94C601F0000E011600500E
:103DCE00011004E0010E915F000E925B93A539D0B5
:103DDE0093A312D093A103D02D0E886F02D02B0E79
:103DEE00886F7FC6E1FF80C6E2FF88C6E6FF7F4B85
:103DFE00802B9F4BA02B0CD093A10AD07FC6E1FF46
:103E0E0080C6E2FF200EE66E7F4B802B9F4BA02BD1
:103E1E00800E006E800E9219005C02E19151000836
:103E2E000FE27FC6E1FF80C6E2FF300EE66E7F4BEB
:103E3E00802B9F4BA02B010E915F000E925BE8D75B
:103E4E003AD093B718D0800E006E800E9219005C97
:103E5E0002E1915100080FE27FC6E1FF80C6E2FF4A
:103E6E00200EE66E7F4B802B9F4BA02B010E915F99
:103E7E00000E925BE8D793A312D093A103D02D0E20
:103E8E00896F02D02B0E896F7FC6E1FF80C6E2FFDD
:103E9E0089C6E6FF7F4B802B9F4BA02B0CD093A1A6
:103EAE000AD07FC6E1FF80C6E2FF200EE66E7F4B92
:103EBE00802B9F4BA02B90C600F0900700524CE039
:103ECE0090C600F0000E016E026E036E003600907A
:103EDE0001360236033600360090013602360336BE
:103EEE00080E0024F66E960E0120F76E000E0220CC
:103EFE00F86E0900F5CF04F00900F5CF05F00900C2
:103F0E00F5CF06F00900F5CF07F09BC600F09CC672
:103F1E0001F09DC602F09EC603F0DDEC0CF00A0E19
:103F2E00046E000E056E066E076EDDEC0CF008C01A
:103F3E0000F009C001F00AC002F00BC003F0300E11
:103F4E0000267FC6E1FF80C6E2FF00C0E6FF7F4B82
:103F5E00802B9F4BA02BAFD7800E006E800E9A1930
:103F6E00005C02E1995100080FE27FC6E1FF80C6B6
:103F7E00E2FF300EE66E7F4B802B9F4BA02B010E87
:103F8E00995F000E9A5BE8D7800E000A006E800ED5
:103F9E008F19005C02E18E51080803E2080E906F43
:103FAE0002D08EC690F690518E5F000E8F5B9053AE
:103FBE0003E194B701D00AD07FC6E1FF80C6E2FFCD
:103FCE002E0EE66E7F4B802B9F4BA02B90C6A7F636
:103FDE0041EC07F095C604F096C605F097C606F0BC
:103FEE0098C607F07AEC04F0BCEC0EF000C09BF61D
:103FFE0001C09CF602C09DF603C09EF690534DE0A4
:10400E00900790C600F0000E016E026E036E003631
:10401E000090013602360336003600900136023625
:10402E000336080E0024F66E960E0120F76E000E73
:10403E000220F86E0900F5CF04F00900F5CF05F067
:10404E000900F5CF06F00900F5CF07F09BC600F08A
:10405E009CC601F09DC602F09EC603F0DDEC0CF08E
:10406E000A0E046E000E056E066E076EDDEC0CF089
:10407E0008C000F009C001F00AC002F00BC003F046
:10408E00300E00267FC6E1FF80C6E2FF00C0E6FFCD
:10409E007F4B802B9F4BA02BB1D78E518F110FE0F2
:1040AE007FC6E1FF80C6E2FF300EE66E7F4B802BAF
:1040BE009F4BA02B010E8E5F000E8F5BEED793A74A
:1040CE001AD0800E006E800E9219005C02E19151A2
:1040DE00000811E27FC6E1FF80C6E2FF200EE66E09
:1040EE007F4B802B9F4BA02B010E915F000E925B9E
:1040FE0091519211EFE1D4EF14F0C00E9315016EB1
:10410E0094C602F0000E0216000E021802E1000E16
:10411E000118D8A480D093A927D084C6E9FF85C6FC
:10412E00EAFFEECF00F0EECF01F000C0E9FF01C0D4
:10413E00EAFFEECF9BF6EECF9CF6EECF9DF6EECFDE
:10414E009EF684C6E9FF85C6EAFF040EEE24006ED5
:10415E00000EEE20016E84C6E1FF85C6E2FF00C0B0
:10416E00E6FF01C0E6FF2FD084C6E9FF85C6EAFF51
:10417E00EECF00F0EECF01F000C0E9FF01C0EAFF84
:10418E00EECF00F0EECF01F0000E01BEFF0E026E7C
:10419E00036E00C09BF601C09CF602C09DF603C0E4
:1041AE009EF684C6E9FF85C6EAFF020EEE24006E77
:1041BE00000EEE20016E84C6E1FF85C6E2FF00C050
:1041CE00E6FF01C0E6FF800E9E19006E800E005CB9
:1041DE0008E1000E9D5D05E1000E9C5D02E1000E02
:1041EE009B5D18E2030E9313000E9413006A016A8E
:1041FE00026A036A9B51005E9C51015A9D51025AFC
:10420E009E51035A00C09BF601C09CF602C09DF65B
:10421E0003C09EF64ED093A927D084C6E9FF85C66B
:10422E00EAFFEECF00F0EECF01F000C0E9FF01C0D3
:10423E00EAFFEECF9BF6EECF9CF6EECF9DF6EECFDD
:10424E009EF684C6E9FF85C6EAFF040EEE24006ED4
:10425E00000EEE20016E84C6E1FF85C6E2FF00C0AF
:10426E00E6FF01C0E6FF25D084C6E9FF85C6EAFF5A
:10427E00EECF00F0EECF01F000C0E9FF01C0EAFF83
:10428E00EECF9BF6EECF9CF6000E9D6F9E6F84C612
:10429E00E9FF85C6EAFF020EEE24006E000EEE2048
:1042AE00016E84C6E1FF85C6E2FF00C0E6FF01C0D5
:1042BE00E6FF000E8F1902E1000E8E190FE1000EBF
:1042CE00006E9E1908E100509D1905E100509C19E1
:1042DE0002E19B51000A02E18E4B8F2BC00E93150B
:1042EE00006E00C005F0AED0010E906F90510A0A1C
:1042FE0034E090C600F0000E016E026E036E0036C2
:10430E000090013602360336003600900136023632
:10431E000336080E0024F66E960E0120F76E000E80
:10432E000220F86E0900F5CF01F00900F5CF02F07A
:10433E000900F5CF03F00900F5CF04F004509E5D9F
:10434E0008E103509D5D05E102509C5D02E10150C4
:10435E009B5D01E202D0902BC9D782D0010E906FE7
:10436E009051080A34E090C600F0000E016E026E05
:10437E00036E00360090013602360336003600908A
:10438E00013602360336E40E0024F66E960E012038
:10439E00F76E000E0220F86E0900F5CF01F009004D
:1043AE00F5CF02F00900F5CF03F00900F5CF04F0C8
:1043BE0004509E5D08E103509D5D05E102509C5D39
:1043CE0002E101509B5D01E202D0902BC9D748D08B
:1043DE00010E906F90510C0A34E090C600F0000E62
:1043EE00016E026E036E0036009001360236033601
:1043FE0000360090013602360336D30E0024F66ED8
:10440E00940E0120F76E000E0220F86E0900F5CF13
:10441E0001F00900F5CF02F00900F5CF03F0090015
:10442E00F5CF04F004509E5D08E103509D5D05E15B
:10443E0002509C5D02E101509B5D01E202D0902B87
:10444E00C9D70ED00550000AD8B44ED70550C00AB1
:10445E00D8B44AD70550800A81E00550400AB8E02A
:10446E00800E006E800E8F19005C02E18E51905D01
:10447E0003E28EC690F60DD0800E8F19006E800E60
:10448E00005C02E190518E5D04E290C68EF6000E45
:10449E008F6F915192110EE0030E9315006E94C61C
:1044AE0001F0000E01160050011004E0010E915FA4
:1044BE00000E925B800E8F19006E800E9219005CBA
:1044CE0002E191518E5D05E28E51915F8F51925BAB
:1044DE0002D0916B926BC40E9315016E9451080B22
:1044EE00026E0250080A02E1400E011808E19151D5
:1044FE00921104E0010E915F000E925B1CD0C00E73
:10450E009315016E9451080B026E0250080A02E1D7
:10451E00800E011810E1800E006E800E9219005C64
:10452E0002E19151020805E2020E915F000E925BCC
:10453E0002D0916B926B93A55DD093A312D093A1F1
:10454E0003D02D0E8A6F02D02B0E8A6F7FC6E1FF2D
:10455E0080C6E2FF8AC6E6FF7F4B802B9F4BA02BC7
:10456E0034D093A10BD07FC6E1FF80C6E2FF200EB0
:10457E00E66E7F4B802B9F4BA02B27D0C00E931542
:10458E00016E9451080B026E0250080A02E1800E71
:10459E0001181BE17FC6E1FF80C6E2FF300EE66E1A
:1045AE007F4B802B9F4BA02B93AB03D0580E8B6F62
:1045BE0002D0780E8B6F7FC6E1FF80C6E2FF8BC6FE
:1045CE00E6FF7F4B802B9F4BA02B9151921111E058
:1045DE007FC6E1FF80C6E2FF300EE66E7F4B802B7A
:1045EE009F4BA02B010E915F000E925B9151921189
:1045FE00EFE174D09151921113E093B711D07FC6B1
:10460E00E1FF80C6E2FF200EE66E7F4B802B9F4BB4
:10461E00A02B010E915F000E925B91519211EFE172
:10462E0093A312D093A103D02D0E8C6F02D02B0E1C
:10463E008C6F7FC6E1FF80C6E2FF8CC6E6FF7F4B24
:10464E00802B9F4BA02B0CD093A10AD07FC6E1FFED
:10465E0080C6E2FF200EE66E7F4B802B9F4BA02B79
:10466E00C00E9315016E9451080B026E0250080A8B
:10467E0002E1400E01180BE17FC6E1FF80C6E2FFAA
:10468E00300EE66E7F4B802B9F4BA02B27D0C00E9B
:10469E009315016E9451080B026E0250080A02E146
:1046AE00800E01181BE17FC6E1FF80C6E2FF300ECF
:1046BE00E66E7F4B802B9F4BA02B93AB03D0580EF7
:1046CE008D6F02D0780E8D6F7FC6E1FF80C6E2FF40
:1046DE008DC6E6FF7F4B802B9F4BA02B800E006E6E
:1046EE00800E8F19005C02E18E51905D0BE27FC649
:1046FE00E1FF80C6E2FF300EE66E7F4B802B9F4BB4
:10470E00A02BECD78EC600F08FC601F0010E8E5F87
:10471E00000E8F5B00500110D8B42AD1C00E931535
:10472E00006E00C0A1F60AD18EC600F08FC601F051
:10473E00000E8FBFFF0E026E036E00360090013624
:10474E000236033600360090013602360336080E66
:10475E000024F66E960E0120F76E000E0220F86E03
:10476E000900F5CF04F00900F5CF05F00900F5CFEB
:10477E0006F00900F5CF07F09BC600F09CC601F0CD
:10478E009DC602F09EC603F0DDEC0CF00A0E046E20
:10479E00000E056E066E076EDDEC0CF008C000F024
:1047AE0009C001F00AC002F00BC003F0300E002465
:1047BE00906FD3D093AB45D08EC600F08FC601F06C
:1047CE00000E8FBFFF0E026E036E00360090013694
:1047DE000236033600360090013602360336E40EFA
:1047EE000024F66E960E0120F76E000E0220F86E73
:1047FE000900F5CF04F00900F5CF05F00900F5CF5B
:10480E0006F00900F5CF07F09BC600F09CC601F03C
:10481E009DC602F09EC603F0DDEC0CF00F0E0016E6
:10482E00000E0116021603167C0E0024F66E980E6C
:10483E000120F76E000E0220F86E0900F5CF90F6FB
:10484E0044D08EC600F08FC601F0000E8FBFFF0E53
:10485E00026E036E003600900136023603360036C5
:10486E000090013602360336E40E0024F66E960EE4
:10487E000120F76E000E0220F86E0900F5CF04F04D
:10488E000900F5CF05F00900F5CF06F00900F5CFC8
:10489E0007F09BC600F09CC601F09DC602F09EC6B6
:1048AE0003F0DDEC0CF00F0E0016000E01160216D2
:1048BE0003166B0E0024F66E980E0120F76E000E96
:1048CE000220F86E0900F5CF90F647D08EC600F0A4
:1048DE008FC601F0000E8FBFFF0E026E036E003604
:1048EE00009001360236033600360090013602364D
:1048FE000336D30E0024F66E940E0120F76E000ED2
:10490E000220F86E0900F5CF04F00900F5CF05F08E
:10491E000900F5CF06F00900F5CF07F09BC600F0B1
:10492E009CC601F09DC602F09EC603F0DDEC0CF0B5
:10493E00070E0014906F300E90270FD0A151000A71
:10494E00D8B4F2D6A151C00AD8B4EED6A151800A7D
:10495E00D8B430D7A151400AB9E07FC6E1FF80C676
:10496E00E2FF90C6E6FF7F4B802B9F4BA02BCAD653
:10497E0093A71AD0800E006E800E9219005C02E191
:10498E009151000811E27FC6E1FF80C6E2FF200EC2
:10499E00E66E7F4B802B9F4BA02B010E915F000E7E
:1049AE00925B91519211EFE1D4EF14F09FC600F09B
:0649BE00A0C601F012008A
:1049C4007FC600F00032009E0032009E0032009E3E
:1049D4000032009E0A0E0002F3CF01F00F0E060112
:0A49E4007F15006E0150002612003E
:1049EE007FC6F6FF80C6F7FF81C6F8FF0900F5CF38
:1049FE0000F0005212E07FC6F6FF80C6F7FF81C6B8
:104A0E00F8FF0900F5CFADF6DAEC00F0010E060165
:104A1E007F27000E80238123E3D71A0E0D6E0D2EF5
:064A2E00FED7000012009B
:104A3400020E0C6E9D0E0D6E0D2EFED70C2EFCD7A5
:064A44000000000012005A
:104A4A000B0E0C6E570E0D6E0D2EFED70C2EFCD7CC
:064A5A0000000000120044
:0A4A6000050E0D6E0D2EFED712009C
:104A6A00020E0C6E080E0D6E0D2EFED70C2EFCD704
:044A7A000000120026
:104A7E00750E0601796F060E7A6F70C67FF671C6D7
:104A8E0080F672C681F673C682F674C683F6790E08
:104A9E00846F060E856FCFEC14F000C077F601C060
:104AAE0078F600507025E16E01507121E26EE66AD3
:0A4ABE0077C600F078C601F0120080
:104AC8000900F5CFE6FF0006FBE10106F9E1120057
:104AD800520E0B6E2B0E0C6E000E0D6E0D2EFED7A9
:0C4AE8000C2EFCD70B2EFAD70000120099
:104AF4000601706B716B800E7119006E800E005C84
:104B040002E1080E705D1AE27051010F7F6F806B35
:104B1400816B826B836B846B856B866B876B886B15
:104B2400896B8A6B8B6B14EC11F06A0E0D6E0D2E73
:104B3400FED700000601704B712BDDD77F6B806BB5
:104B4400816B826B836B846B856B866B876B886BE5
:104B5400896B8A6B8B6B14EC11F00A0E06017F6F64
:104B6400806B816B826B836B846B856B866B876BCD
:0E4B7400886B896B8A6B8B6B14EC11F012004E
:104B8200000E0B6E010E0C6E066A076A066A076A51
:104B9200800E0718006E800E005C02E10C0E065CAF
:104BA200D8B08DD0065006017025E96E07507121EC
:104BB200EA6EEECF01F001C00AF001503B0A02E1B9
:104BC200200E0A6E0A50B00A2EE1046A056A800EAF
:104BD2000518006E800E005C02E1080E045C22E201
:104BE200C20E0424E96E000E0520EA6E030E026E68
:104BF20006C000F007C001F0025005E00036009048
:104C02000136FF0FFAD7045000260550012200504A
:104C12000B24E16E01500C20E26EEECFE6FF044A57
:104C2200052AD5D749D0030E006E0AC008F0000E3F
:104C3200096E005005E0083608900936FF0FFAD7D2
:104C4200046A056A800E0518006E800E005C02E19F
:104C5200080E045C31E204500824006E055009205D
:104C6200016E1A0E0024F66E850E0120F76E000EFC
:104C7200F86E000E01BEFF0EF8220900F5CF03F018
:104C8200030E026E06C000F007C001F0025005E0FC
:104C9200003600900136FF0FFAD704500026055067
:104CA200012200500B24E16E01500C20E26E03C081
:104CB200E6FF044A052AC6D7064A072A69D7120020
:104CC2003A0E0501396F0A0E3A6F000E3B6F000E65
:104CD2003C6F300E356F140E366F000E376F000EBC
:104CE200386FC80E3D6F140E3E6F000E3F6F000E00
:104CF200406F220E456F150E466FA70E476F060EC8
:104D0200486FEE0E416F150E426FA70E436F060EEF
:104D1200446FA60E496F1C0E4A6F000E4B6F000EB9
:104D22004C6F949894968B988B9694889486C79E91
:084D3200C79C380EC66E12008A
:104D3A0018EC0AF0D00E0601A76FF7EC0AF006018C
:104D4A00A76BF7EC0AF064EC0AF0D10E0601A76F24
:104D5A00F7EC0AF0010E0601A76F91EC0AF000C009
:104D6A0068F500C07FF629DE00C065F5010EA76F61
:104D7A0091EC0AF000C0FEF000C07FF61EDE00C013
:104D8A006AF5010EA76F91EC0AF000C0EDF0010E72
:104D9A000601A76F91EC0AF0070E0014016E01C01C
:104DAA00FCF00150070802E20001FC6B010E06014B
:104DBA00A76F91EC0AF000C0EEF0010E0601A76F92
:104DCA0091EC0AF01F0E00140001FB6F0601A76B9D
:104DDA0091EC0AF000C0FDF053EC0EF0FBC07FF638
:104DEA00ECDD00C0ECF000500C0802E20001EC6BB4
:104DFA00EDC07FF6B10E0601806F000E816FF9ECEF
:104E0A0011F03A0E0001B36FFEC07FF6B40E060130
:104E1A00806F000E816FF9EC11F03A0E0001B66F47
:104E2A0068C57FF6B70E0601806F000E816FF9EC38
:104E3A0011F00001B96BEEC07FF6A60E0601806F75
:104E4A00000E816FF9EC11F02D0E0001A86FFBC066
:104E5A007FF6A90E0601806F000E816FF9EC11F042
:104E6A002D0E0001AB6FFDC07FF6AC0E0601806F00
:104E7A00000E816FF9EC11F00001AE6B0601705162
:104E8A00010A1DE1A60E7F6F000E806FE1EC11F0A2
:104E9A002C0E06017F6F9A0E806F000E816FA2DDC5
:104EAA00B10E06017F6F000E806FE1EC11F02C0E3F
:104EBA0006017F6F9A0E806F000E816F93DD1200DC
:104ECA00090E0B6E1E0E0C6EE40E0D6E0D2EFED725
:104EDA000C2EFCD70B2EFAD700008B820F0E060180
:104EEA007F6F806B816B826B836B846B856B866B48
:104EFA00876B886B896B8A6B8B6B14EC11F00B0ECA
:104F0A0006017F6F070E806F070E816F070E826F93
:104F1A00070E836F070E846F070E856F070E866F65
:104F2A00070E876F070E886F070E896F070E8A6F45
:104F3A00070E8B6F14EC11F08996090E06017F6F2C
:104F4A00806B816B826B836B846B856B866B876BE3
:104F5A00886B896B8A6B8B6B14EC11F00A0E060155
:104F6A007F6F806B816B826B836B846B856B866BC7
:104F7A00876B886B896B8A6B8B6B14EC11F00C0E48
:104F8A0006017F6F010E806F010E816F010E826F25
:104F9A00010E836F010E846F010E856F010E866FFD
:104FAA00010E876F010E886F010E896F010E8A6FDD
:104FBA00010E8B6F14EC11F0D00E0C6EC90E0D6E33
:0E4FCA000D2EFED70C2EFCD7000000001200AA
:104FD8000601706B716B000E0001D76F010ED86F60
:104FE8000601706B716B800E7119006E800E005C8B
:104FF80002E1080E705DD8B0C4D07051010F7F6F08
:10500800580E0001D725006E000ED821016E06014A
:1050180070510024E96E71510120EA6EEECF80F6DE
:10502800500E0001D725006E000ED821016E060132
:1050380070510024E96E71510120EA6EEECF81F6BD
:10504800480E0001D725006E000ED821016E06011A
:1050580070510024E96E71510120EA6EEECF82F69C
:10506800400E0001D725006E000ED821016E060102
:1050780070510024E96E71510120EA6EEECF83F67B
:10508800380E0001D725006E000ED821016E0601EA
:1050980070510024E96E71510120EA6EEECF84F65A
:1050A800300E0001D725006E000ED821016E0601D2
:1050B80070510024E96E71510120EA6EEECF85F639
:1050C800280E0001D725006E000ED821016E0601BA
:1050D80070510024E96E71510120EA6EEECF86F618
:1050E800200E0001D725006E000ED821016E0601A2
:1050F80070510024E96E71510120EA6EEECF87F6F7
:10510800180E0001D725006E000ED821016E060189
:1051180070510024E96E71510120EA6EEECF88F6D5
:10512800100E0001D725006E000ED821016E060171
:1051380070510024E96E71510120EA6EEECF89F6B4
:10514800080E0001D725006E000ED821016E060159
:1051580070510024E96E71510120EA6EEECF8AF693
:1051680070510001D725E96E060171510001D8215F
:10517800EA6EEECF8BF614EC11F00601704B712B32
:0451880032D7120008
:10518C00020E0601706F000E716FEEEC13F006014B
:10519C00746B756BA00E0001C025E16E050EC1216C
:1051AC00E26EE66A000EC15D02E1160EC05DD8B07B
:1051BC0008D1000E006EC151005C02E1C051130811
:1051CC00D8B0FFD0020E0601726F000E736F000193
:1051DC00C1510601735D04E10001C0510601725D0D
:1051EC002FE2A00E7225E96E050E7321EA6EEE50C9
:1051FC003B0A23E1A00E7225E16E050E7321E26ECF
:10520C00E66AEF0E7425786F000E7521796FA00E8B
:10521C0070257F6F050E7121806FF9EC13F078C645
:10522C00E1FF79C6E2FF00C0E6FF744B752B010E5F
:10523C007225706F000E7321716F724B732BC7D771
:10524C00F2C076F6000E776FF4C0F2F0F3C0F4F013
:10525C0076C6F3F0EFC0EEF01F0E0001F015FB6FF9
:10526C00F1C0FDF0F2C0FCF0FBC07FF6E2EC24F0E4
:10527C0000C0ECF00001EC510C08D8A0EC6B81B232
:10528C003DD0F40E06017F6F980E806F000E816F7B
:10529C00F7EC24F0FCC07FF6000E0601806F9F0E29
:1052AC00816F040E826F5FEC13F0090EAD6FDAECB8
:1052BC0000F09F0E06017F6F040E806F62EC14F0FD
:1052CC00090EAD6FDAEC00F0030E006E000E016EED
:1052DC00FCC004F0000E056E99EC10F0490E002491
:1052EC00E96E000E0120EA6EEECF7FF6EECF80F66F
:1052FC00EECF81F6F7EC24F0EEEC13F00001FC514C
:10530C0007080AE2FC6BA00E06017F6F960E806FF9
:10531C00000E816FF7EC24F0F3C0EDF0F4C0FEF05A
:10532C0006017F6B806B03EC11F0FEC07FF6DCECAA
:10533C0010F000C080F6010E7F6F03EC11F0EDC091
:10534C007FF6DCEC10F000C080F6020E7F6F03ECF1
:10535C0011F0030E06017F6FFCC080F603EC11F018
:10536C00EEC07FF6DCEC10F000C080F6040E7F6F10
:10537C0003EC11F0FBC07FF6DCEC10F000C080F603
:10538C00050E7F6F03EC11F0FDC07FF6DCEC10F026
:10539C0000C080F6060E7F6F03EC11F0070E0601BD
:1053AC007F6F100E806F03EC11F05F0E06017F6FA4
:1053BC00970E806F000E816FF7EC24F0EEEC13F07B
:1053CC0012D0050E06017F6F940E806F000E816F58
:1053DC00F7EC24F0FA0E06017F6F910E806F000E31
:0853EC00816FF7EC24F01200C0
:1053F40006017F6B20EC12F000C068F5010E7F6F90
:1054040020EC12F000C0FEF0020E7F6F20EC12F0D0
:1054140000C0EDF0030E7F6F20EC12F0070E0014B5
:10542400016E01C0FCF00150070802E20001FC6BB0
:10543400040E06017F6F20EC12F000C0EEF0050EA2
:105444007F6F20EC12F01F0E00140001FB6F060E9C
:1054540006017F6F20EC12F000C0FDF0FBC07FF668
:10546400E2EC24F000C0ECF000500C0802E2000171
:04547400EC6B1200CB
:10547800A6A202D00000FCD7A69C71C6AAFF70C6DF
:10548800A9FF72C6A8FFA69EA684F2CF00F0F29EDE
:10549800550EA76EAA0EA76EA68200BE02D0F29E77
:1054A80001D0F28EA694A1B802D00000FCD7A19832
:0254B8001200E0
:1054BA00040E0001636F060E646F6251000AD8A4DD
:1054CA00BFD10601706B716B800E7119006E800E70
:1054DA00005C02E1600E705D0AE2040E7025E16E66
:1054EA00060E7121E26EE66A704B712BEDD7040E3F
:1054FA000001636F060E646F040EBA6F060EBB6F6F
:10550A00BAC0E1FFBBC0E2FF200EE66E010EBA256B
:10551A0006017F6F000E0001BB210601806FB10EEC
:10552A00816F000E826F080E836F000E846FF4EC99
:10553A0012F0090E0001BA25E16E000EBB21E26EDF
:10554A003B0EE66E0A0EBA25006E000EBB21016EF6
:10555A0000C0BEF001C0BFF000C07FF601C080F6F7
:10556A00030E006E000E016EFCC004F0000E056E04
:10557A0099EC10F0490E0024E96E000E0120EA6E43
:10558A00EECF81F6EECF82F6EECF83F6A6EC14F0DC
:10559A00BEC07FF6BFC080F6C4EC11F000C070F642
:1055AA0001C071F600500001BE25E16E0150BF2115
:1055BA00E26E200EE66E060170510001BE25006EF5
:1055CA00060171510001BF21016E00C0BCF001C08B
:1055DA00BDF000C0E1FF01C0E2FFA6C0E6FF010E78
:1055EA00BC25E16E000EBD21E26EA7C0E6FF020EE9
:1055FA00BC25E16E000EBD21E26E200EE66E030EA2
:10560A00BC25006E000EBD21016E00C091F001C0E4
:10561A0092F000C07FF601C080F6030E006E000E05
:10562A00016EECC004F0000E056E99EC10F06A0EE3
:10563A000024E96E000E0120EA6EEECF81F6EECF6D
:10564A0082F6EECF83F6A6EC14F091C07FF692C0F4
:10565A0080F6C4EC11F000C070F601C071F600507B
:10566A0000019125E16E01509221E26E200EE66E54
:10567A000601705100019125006E06017151000169
:10568A009221016E00C093F001C094F000C0E1FFC6
:10569A0001C0E2FF320EE66E010E9325E16E000EA6
:1056AA009421E26E300EE66E020E9325E16E000E34
:1056BA009421E26EACC0E6FF030E9325E16E000E64
:1056CA009421E26EADC0E6FF040E9325E16E000E52
:1056DA009421E26E3B0EE66E050E9325006E000ED7
:1056EA009421016E00C097F001C098F000C07FF6C7
:1056FA0001C080F6220E0601816F9A0E826F000E9B
:10570A00836FA6EC14F0710E06017F6F050E806F91
:10571A00C4EC11F0010E005C026E000E0158036E1B
:10572A0002C070F603C071F6040E00019725006EE0
:10573A00000E9821016E00C097F001C098F000C0D9
:10574A007FF601C080F6720E0601816F050E826F28
:10575A0002C083F603C084F6F4EC12F07051000123
:10576A009725006E0601715100019821016E00C053
:10577A0097F001C098F000C0E1FF01C0E2FFB00E4F
:10578A00E66E010E9725E16E000E9821E26E3B0E41
:10579A00E66E020E9725006E000E9821016E00C07B
:1057AA0095F001C096F000C07FF601C080F6610E48
:1057BA000601816F010E826F38EC13F00A0E0001A8
:1057CA009525006E000E9621016E00C095F001C06D
:1057DA0096F000C0E1FF01C0E2FFB00EE66E010ED6
:1057EA009525E16E000E9621E26E3B0EE66E020EE4
:1057FA009525E16E000E9621E26EE66A0401EF6BD2
:10580A0063C07FF664C080F6C4EC11F000C043F0B8
:10581A0001C044F0800E026E800E0118025C02E1A3
:10582A0000505F0804E25F0E436E000E446E5F0E86
:10583A0000016325E16E000E6421E26EE66A99D0EA
:10584A0005012E6B040E0001636F060E646F0601DC
:10585A00706B716B800E7119006E800E005C02E134
:10586A00600E705D08E263C0E1FF64C0E2FFE66AB1
:10587A00704B712BEFD7040E0001BA6F060EBB6F87
:10588A00BAC0E1FFBBC0E2FF200EE66E010EBA25E8
:10589A0006017F6F000E0001BB210601806FB10E69
:1058AA00816F000E826F080E836F000E846FF4EC16
:1058BA0012F063C07FF664C080F6C4EC11F000C039
:1058CA0070F601C071F6090E0001BA25E16E000EEC
:1058DA00BB21E26E200EE66EEF0E06017F6F040E0C
:1058EA00806FC4EC11F000C070F601C071F60A0EA8
:1058FA000001BA2506017F6F000E0001BB210601D7
:10590A00806FEF0E816F040E826F00C083F601C0B4
:10591A0084F6F4EC12F00A0E0001BA25006E000EAD
:10592A00BB21016E060170510024E16E7151012004
:10593A00E26EE66A63C07FF664C080F6C4EC11F0DA
:10594A0000C043F001C044F0800E026E800E0118C0
:10595A00025C02E100505F0804E25F0E436E000E33
:10596A00446E5F0E00016325E16E000E6421E26E53
:04597A00E66A1200C7
:10597E000601766B776B70C678F671C679F6800E77
:10598E007119006E800E005C02E1000E705D0BE27C
:10599E00010E766F000E776F70510008786F71C62A
:1059AE0079F6000E795778C67FF679C680F672C6FC
:1059BE0081F673C682F65FEC13F0060E746F000E5E
:1059CE00756F000E006E7551005C02E17451000897
:1059DE0019E274517225E16E75517321E26E010E5A
:1059EE00745D006E000E7559016E00507225E96EE1
:1059FE0001507321EA6EEECFE6FF010E745F000ECA
:105A0E00755BDFD772C6E1FF73C6E2FF200EE66E4E
:105A1E00765177111AE0746B756B74517225E96EBD
:105A2E0075517321EA6EEE50200A03E1744B752B0B
:105A3E00F4D7010E745F000E755B74517225E16E22
:0C5A4E0075517321E26E2D0EE66E120001
:105A5A006300A0FF32F5630080FFFFF00101D890D8
:105A6A005837503748374037383730372837203794
:105A7A001837103708370037D89059375137493710
:105A8A00413739373137293721371937113709372C
:105A9A000137D8905A3752374A3742373A3732376E
:105AAA002A3722371A3712370A370237D8905B3724
:105ABA0053374B3743373B3733372B3723371B376C
:105ACA0013370B370337D8905C3754374C37443782
:105ADA003C3734372C3724371C3714370C37043704
:105AEA00D8905D3755374D3745373D3735372D37E0
:105AFA0025371D3715370D370537D8905E37563796
:105B0A004E3746373E3736372E3726371E37163743
:105B1A000E370637D8905F3757374F3747373F37F3
:105B2A0037372F3727371F3717370F3707376000B1
:0C5B3A00FCF3E0FF6100C8F4E8FF12007B
:105B46000601726B736B70C603F071C604F070C603
:105B560005F071C606F003C0E9FF04C0EAFFEE5087
:105B6600200A04E17251731101E110D0010E726F27
:105B7600000E736F03C0E9FF04C0EAFF05C0E1FF32
:105B860006C0E2FFEECFE6FF054A062A03C001F093
:105B960004C002F0034A042A01C0E9FF02C0EAFF7A
:105BA600EE50000AD8E170C600F071C601F012008E
:105BB6000001C06BC16B000EC15D02E1630EC05DEA
:105BC60012E2A00EC025E16E050EC121E26EE66A64
:105BD600010EC025006E000EC121016E00C0C0F08E
:105BE60001C0C1F0E8D76B86CA6BCB6BC06BC16BCB
:105BF6009EAA02D0AECFCEF0CE6BCC6BCD6B06019B
:0A5C06006C6B6D6B9D8AF28E12002C
:105C100070C6F6FF71C6F7FF72C6F8FF0900F5CF30
:105C200000F0005212E070C6F6FF71C6F7FF72C6B0
:105C3000F8FF0900F5CFADF6DAEC00F0010E060131
:105C40007027000E71237223E3D71A0E0D6E0D2EEE
:065C5000FED70000120067
:105C560070C674F671C675F674C67FF675C680F69C
:105C6600E4EC13F000C076F6060174517225016E5D
:105C760075517321026E7051015CE16E71510258CB
:105C8600E26E00C0E6FF7651000A01E119D0020E6D
:105C96000B6EA00E0C6E920E0D6E0D2EFED70C2EF8
:105CA600FCD70B2EFAD70000744B752B800E751996
:105CB600006E800E030A005C02E1FF0E745DCCE309
:105CC60074517225006E75517321016E7051005C1E
:0C5CD600E16E71510158E26EE66A1200A6
:105CE2003F0E806E0F01386B230E926E9294898460
:105CF2009296899692988988796A786A546BFF0E8F
:105D0200816EFF0E936E396BFF0E616E93849382E8
:105D1200F19EFF0E826E3A6B948E948C546B949A21
:105D22008B8A9492949094948B828B948B90606AD9
:025D320012005D
:105D3400B40E0501616F010E626FAD0E636F060E46
:105D4400646FFF0E5D6FFF0E5E6F000E5F6F000EDF
:105D5400606FFF0E516FFF0E526F000E536F000EF7
:105D6400546FFF0E4D6FFF0E4E6F000E4F6F000EFF
:105D7400506FAC8A900EAB6E948E949C9EAA03D006
:085D8400AECF00F0FBD71200C6
:105D8C00D09EF18C9F8A9F809D8A9D80F28CF28E92
:025D9C001200F3
:105D9E0000C008F00150006E016A026A036A0B6AC5
:105DAE000C6A016A026A036A960E036E0A6A00AEF4
:105DBE00E7EF2EF0081E001E082AD8B4002A0A8E1D
:105DCE0000C001F008C000F0086A026AA8EC13F0E7
:025DDE001200B1
:105DE00072C601F0010E006E015004E00036009012
:105DF000FF0FFBD700C076F6001C0601756F746BB1
:105E000070C6E9FF71C6EAFF736B7351070824E39C
:105E10007551EF16120EE9267551EF1630EC25F08C
:105E20007651EF1230EC25F0120EE95E7651EF1448
:105E3000006E0CE073C601F0010E006E015004E02C
:105E400000360090FF0FFBD70050741335EC25F09F
:0E5E500035EC25F0732BD9D774C600F0120084
:105E5E0070C600F00032009E0032009E0032009E9E
:105E6E000032009E9D0E0024F66E980EF76E000E08
:105E7E00F722000EF86E000EF8220900F5CF00F0A2
:105E8E0071C6E1FF72C6E2FF00C0E6FF010E060119
:105E9E007125E16E000E7221E26E0F0E7015006E0E
:105EAE009D0E0024F66E980EF76E000EF722000E71
:105EBE00F86E000EF8220900F5CF00F000C0E6FFE4
:105ECE00020E7125E16E000E7221E26EE66A12007C
:105EDE0006017A6B71AF0DD02D0E7A6F72C6E1FF8F
:105EEE0073C6E2FF2D0EE66E701F711F704B712B85
:105EFE0008D02B0E7A6F72C6E1FF73C6E2FF2B0E2F
:105F0E00E66E70C600F071C601F001320032019EDD
:105F1E0001320032019E01320032019E0132003206
:105F2E00019E00C074F601C075F6010E72257B6FDE
:105F3E00000E73217C6F0A0E046E000E056EC1EC0E
:105F4E0010F00A0E046E000E056EC1EC10F008C0C3
:105F5E0000F009C001F0300E00267BC6E1FF7CC6C2
:105F6E00E2FF00C0E6FF020E72257B6F000E73216A
:105F7E007C6F0A0E046E000E056E74C600F075C6B8
:105F8E0001F0C1EC10F008C000F009C001F0300EB5
:105F9E0000267BC6E1FF7CC6E2FF00C0E6FF70C6AE
:105FAE0076F671C677F6000E786F796F0F0E76174C
:105FBE00000E771778177917080E7225E16E000E0E
:105FCE007321E26EE66A76C600F077C601F078C6F7
:105FDE0002F079C603F0710E046E020E056E000E0D
:105FEE00066E076E7DEC14F000C076F601C077F6F3
:105FFE0002C078F603C079F6030E7225E16E000E2C
:10600E007321E26E2E0EE66E040E72257B6F000E6D
:10601E0073217C6FE80E046E030E056E000E066E85
:10602E00076E76C600F077C601F078C602F079C624
:10603E0003F047EC12F0300E00267BC6E1FF7CC663
:10604E00E2FF00C0E6FF050E060172257B6F000E13
:10605E0073217C6F640E046E000E056E066E076E65
:10606E0076C600F077C601F078C602F079C603F066
:10607E0047EC12F00A0E046E000E056E066E076EE9
:10608E0047EC12F008C000F009C001F00AC002F09F
:10609E000BC003F0300E00267BC6E1FF7CC6E2FF8C
:1060AE0000C0E6FF060E06017225E16E000E73219A
:1060BE00E26EE66A74C600F075C601F0000E026E5E
:1060CE00036EE80E046E030E056E000E066E000ED5
:1060DE00076E7DEC14F000C07BF601C07CF602C0AA
:1060EE007DF603C07EF60A0E046E000E056E066E79
:1060FE00076E76C600F077C601F078C602F079C654
:10610E0003F047EC12F0005006017B25686F01503A
:10611E007C21696F02507D216A6F03507E216B6F67
:10612E007A512D0A14E1006A016A026A036A685103
:10613E00005E6951015A6A51025A6B51035A00C0EE
:10614E0068F601C069F602C06AF603C06BF67AC63D
:04615E0000F012003B
:1061620072C601F0010E006E015004E0003600908C
:10617200FF0FFBD700C074F6001E70C6E9FF71C6A0
:10618200EAFF0050EF16120EE9260050EF1625EC3A
:1061920025F006017451EF12120EE95E1AEC25F099
:1061A2007451EF14736F7351000A000ED8A4010EDC
:0C61B200736F25EC25F073C600F012009E
:1061BE00060E0C6E300E0D6E0D2EFED70C2EFCD76D
:0461CE0000001200BB
:1061D20072C601F0010E006E015004E0003600901C
:1061E200FF0FFBD700C076F6001E00C075F670C622
:1061F200E9FF71C6EAFF0050EF16120EE92606010A
:10620200746B7451070816E374C600F073C601F08C
:10621200005004E00132019EFF0FFBD77551EF16CB
:1062220001A002D07651EF121AEC25F07651EF124E
:10623200742BE7D7120EE95E35EC25F035EC25F02C
:02624200120048
:1062440018EC4DF09B6A700ED36E9B8CD26AD3B45B
:1062540001D0FDD7290E0B6E960E0C6E7F0E0D6EBF
:106264000D2EFED70C2EFCD70B2EFAD738DD520E8E
:106274000B6E2B0E0C6E000E0D6E0D2EFED70C2E1B
:10628400FCD70B2EFAD700008B948B820A0E0001E8
:10629400656F000E666F89980501339F3481010193
:1062A400606B060E0001676F626BB886030EB06EFA
:1062B400400EAF6EAC843CDD090E0B6E1E0E0C6EF0
:1062C400E40E0D6E0D2EFED70C2EFCD70B2EFAD736
:1062D40000000C0E0601AD6FDAEC00F0090E0B6E37
:1062E4001E0E0C6EE40E0D6E0D2EFED70C2EFCD77A
:1062F4000B2EFAD70000EEEC13F00001616B040ED4
:10630400636F060E646F0501306B316B000E315DF7
:1063140002E1630E305D0AE2040E3025E16E060EE2
:106324003121E26EE66A304B312BF0D7306B316BA2
:10633400000E315D02E13F0E305D0AE2EF0E3025C2
:10634400E16E040E3121E26EE66A304B312BF0D758
:106354002E6B306B316B000E315D02E1800E305DCF
:106364000AE29F0E3025E16E010E3121E26EE66AEB
:10637400304B312BF0D7040E0001636F060E646FAF
:10638400000ED76F010ED86F0501306B316B030E11
:10639400315D02E1000E305D0AE29F0E3025E16EB0
:1063A400010E3121E26EE66A304B312BF0D7EEEC70
:1063B40013F0EADCDBEC2DF0010E1B6E0501306BF3
:1063C400316B000E315D02E10D0E305D1BE2030EF8
:1063D400006E000E016E30C504F031C505F099EC75
:1063E40010F01C0E0024E96E000E0120EA6EEECFC0
:1063F40070F6EECF71F6EECF72F608DC0501304B85
:10640400312BDFD7090E0B6E1E0E0C6EE40E0D6ED3
:106414000D2EFED70C2EFCD70B2EFAD70000EEEC77
:1064240013F0EEEC13F0040E0001636F060E646FBC
:10643400410E0601706F970E716F000E726F08ECBB
:106444002EF00601706B716B63C072F664C073F654
:1064540000DC020E0B6EA00E0C6E920E0D6E0D2E55
:10646400FED70C2EFCD70B2EFAD7000063C07FF6A4
:1064740064C080F662EC14F0EEEC13F0900E0601AA
:10648400706F000E716F63C072F664C073F62BEC0C
:106494002EF063C07FF664C080F662EC14F0060E42
:1064A40000016325E16E000E6421E26EE66A040ECB
:1064B400632506017F6F000E000164210601806FD1
:1064C400F9EC13F000C0DAF0090E00016325E16E67
:1064D400000E6421E26EE66A070E632506017F6FF3
:1064E400000E000164210601806FF9EC13F000C076
:1064F400D9F0020E0B6EA00E0C6E920E0D6E0D2EC8
:10650400FED70C2EFCD70B2EFAD70000A00E706F0E
:10651400000E716F63C072F664C073F62BEC2EF03C
:1065240063C07FF664C080F662EC14F0060E0001CE
:106534006325E96E000E6421EA6E300EEE5C006E97
:10654400016A000E015A0A0E046E000E056E99ECE3
:1065540010F000C065F001C066F0070E6325E96E17
:10656400000E6421EA6E300EEE5C026E036A000EC9
:10657400035A02500024656F03500120666F020E17
:106584000B6EA00E0C6E920E0D6E0D2EFED70C2E01
:10659400FCD70B2EFAD70000196AC00E0601706FE3
:1065A400000E716F63C072F664C073F62BEC2EF0AC
:1065B40063C07FF664C080F662EC14F0040E000140
:1065C4006325E96E000E6421EA6E300EEE5C196EEE
:1065D4000A0E1902F3CF19F0050E6325E96E000EB9
:1065E4006421EA6E300EEE5C006E005019260F0E28
:1065F4001916CF6BD06BD00E0601706F000E716F41
:1066040063C072F664C073F62BEC2EF063C07FF6A1
:1066140064C080F662EC14F0060E00016325E96E96
:10662400000E6421EA6E300EEE5C006E016A000E0C
:10663400015A640E046E000E056E99EC10F000C051
:106644006EF601C06FF66EC6CFF06FC6D0F0070EBF
:106654006325E96E000E6421EA6E300EEE5C006E76
:10666400016A000E015A0A0E046E000E056E99ECC2
:1066740010F0005006016E250001CF6F0150060195
:106684006F210001D06F080E6325E96E000E6421AE
:10669400EA6E300EEE5C006E016A000E015A005084
:1066A400CF270150D023050E6325E96E000E642127
:1066B400EA6EEE502D0A06E1CF510008CF6FD0519B
:1066C400000ED057800ED019006E800EFE0A005CBA
:1066D40002E1D40ECF5D0BE3800E010A006E800E42
:1066E400D019005C02E1CF512C0801E302D0CF6B3A
:1066F400D06BCFC000F0D0C001F0CFEC2EF0000E74
:10670400046E000E056E480E066E850E076E84EC50
:1067140006F000C0D1F001C0D2F002C0D3F003C033
:10672400D4F0EEEC13F01A6A0001626BEEEC13F095
:106734007C0E0601706F960E716F000E726F08EC7E
:106744002EF00001D56BD66B800E0601706F0F0E14
:10675400716F726B04DD31DD800E706F0F0E716F1F
:10676400726B330E736F33DD28DD800E706F0F0E86
:10677400716F726BF0EC2EF000C0CEF01EDD8D0E4A
:10678400706F980E716F000E726F08EC2EF004019A
:106794009F6BCEC070F69F0E0601716F040E726F70
:1067A4002FEC2FF09F0E7F6F040E806F62EC14F0BD
:1067B400D20E706F990E716F000E726F08EC2EF08E
:1067C4000501306B316B000E315D02E1060E305D68
:1067D40032E2800E0601706F0F0E716F726BF0EC77
:1067E4002EF000C0CEF0D00E0C6EC90E0D6E0D2E24
:1067F400FED70C2EFCD700000000DB0E050130256F
:10680400E16E000E3121E26ECEC0E6FF04019F6B03
:10681400CEC070F69F0E0601716F040E726F2FECDE
:106824002FF09F0E7F6F040E806F62EC14F0050151
:10683400304B312BC8D7CA0E0601706F990E716F99
:10684400000E726F08EC2EF0800E0601706F0F0EB2
:10685400716F726BF0EC2EF000C0CEF004019F6BF0
:10686400CEC070F69F0E0601716F040E726F2FEC8E
:106874002FF09F0E7F6F040E806F62EC14F0EEEC2D
:1068840013F0CE0E0601706F970E716F000E726FCB
:1068940008EC2EF0800E0601706F0F0E716F726B94
:1068A4005EDC800E706F0F0E716F726BCC0E736FA7
:1068B4008EDC800E706F0F0E716F726B440E736FEF
:1068C40086DC110E0B6E3C0E0C6ECB0E0D6E0D2E77
:1068D400FED70C2EFCD70B2EFAD7800E706F0F0E3E
:1068E400716F726B3CDC800E706F0F0E716F726B88
:1068F400CC0E736F6CDC800E706F0F0E716F726B49
:10690400BE0E736F64DC030E0B6E080E0C6E770EF6
:106914000D6E0D2EFED70C2EFCD70B2EFAD7800E43
:10692400706F0F0E716F726BF0EC2EF000C047F0B9
:10693400000E486E800E706F0F0E716F726BF0EC6C
:106944002EF000C003F0026A47500224006E485043
:106954000320016E00C045F001C046F000C070F68F
:1069640001C071F6810E726F010E736F6FEC2FF020
:1069740000C0E9F0810E706F010E716FA3EC2DF071
:10698400810E7F6F010E806FC4EC11F000C0EAF03D
:1069940001C0EBF0810E00247F6F010E0120806F97
:1069A4001D0E816F9A0E826F000E836FA6EC14F099
:1069B400810E06017F6F010E806F62EC14F0EEEC25
:1069C40013F0EEEC13F0610E06017F6F010E806F81
:1069D400BA0E816F990E826F000E836FA6EC14F0CD
:1069E400EEEC13F0040E0001636F060E646F0501F4
:1069F400306B316B000E315D02E1640E305D0AE2F2
:106A0400040E3025E16E060E3121E26EE66A304B4B
:106A1400312BF0D7EEEC13F02E0E0601706F980EAA
:106A2400716F000E726F08EC2EF0280EC86E61ECC8
:106A340026F0990E0601706F970E716F000E726F3B
:106A440008EC2EF00E0E06017F6F400E806F03ECF3
:106A540011F0430E0601706F980E716F000E726F85
:106A640008EC2EF0010E0601706F9DEC26F0EEECA2
:106A740013F0040E0001636F060E646FEA6BEB6B98
:106A84008B908B948B82B60E0601706F920E716F91
:106A9400000E726F08EC2EF07C0E0601706F970EDC
:106AA400716F000E726F08EC2EF065EC27F06CEC41
:106AB40025F0230E0601706F970E716F000E726F32
:106AC40008EC2EF07AEC25F0EEEC13F08B82EEEC71
:106AD40013F0990E0601706F930E716F000E726FB2
:106AE40008EC2EF09F0E06017F6F040E806F010EDE
:106AF400816F990E826F000E836FA6EC14F09F0EC7
:106B04000601706F040E716FC1EC25F0ECEC27F0F8
:106B1400A30E0B6E570E0C6E020E0D6E0D2EFED7CD
:106B24000C2EFCD70B2EFAD70000630E706F930E59
:106B3400716F000E726F08EC2EF0000E0001D76F1B
:106B4400010ED86FD56BD66B000ED65D02E1080E30
:106B5400D55DD8B0B6D0D551010F06017F6F580E60
:106B64000001D725006E000ED821016ED5510024F6
:106B7400E96ED6510120EA6EEECF80F6500ED7258D
:106B8400006E000ED821016ED5510024E96ED65155
:106B94000120EA6EEECF81F6480ED725006E000E76
:106BA400D821016ED5510024E96ED6510120EA6E38
:106BB400EECF82F6400ED725006E000ED821016E6E
:106BC400D5510024E96ED6510120EA6EEECF83F64A
:106BD400380ED725006E000ED821016ED551002441
:106BE400E96ED6510120EA6EEECF84F6300ED72539
:106BF400006E000ED821016ED5510024E96ED651E5
:106C04000120EA6EEECF85F6280ED725006E000E21
:106C1400D821016ED5510024E96ED6510120EA6EC7
:106C2400EECF86F6200ED725006E000ED821016E19
:106C3400D5510024E96ED6510120EA6EEECF87F6D5
:106C4400180ED725006E000ED821016ED5510024F0
:106C5400E96ED6510120EA6EEECF88F6100ED725E4
:106C6400006E000ED821016ED5510024E96ED65174
:106C74000120EA6EEECF89F6080ED725006E000ECD
:106C8400D821016ED5510024E96ED6510120EA6E57
:106C9400EECF8AF6D551D725E96ED651D821EA6EC2
:106CA400EECF8BF614EC11F0150E0C6EC60E0D6EB5
:106CB4000D2EFED70C2EFCD700000001D54BD62B91
:106CC40043D7EEEC13F00001D56BD66B000ED65D06
:106CD40002E1600ED55DD8B087D0ECEC27F06300FC
:106CE400A0FF32F5630080FFFFF00101D890583710
:106CF4005037483740373837303728372037183738
:106D0400103708370037D89059375137493741374A
:106D140039373137293721371937113709370137CF
:106D2400D8905A3752374A3742373A3732372A37A8
:106D340022371A3712370A370237D8905B3753375E
:106D44004B3743373B3733372B3723371B3713370F
:106D54000B370337D8905C3754374C3744373C37BC
:106D640034372C3724371C3714370C370437D89072
:106D74005D3755374D3745373D3735372D3725374F
:106D84001D3715370D370537D8905E3756374E37D0
:106D940046373E3736372E3726371E3716370E37E7
:106DA4000637D8905F3757374F3747373F3737372E
:106DB4002F3727371F3717370F3707376000FCF394
:106DC400E0FF6100C8F4E8FF050E0B6E0F0E0C6EB9
:106DD400F10E0D6E0D2EFED70C2EFCD70B2EFAD70E
:106DE4000001D54BD62B72D7A30E0B6E570E0C6E2B
:106DF400020E0D6E0D2EFED70C2EFCD70B2EFAD7DD
:106E040000007AEC25F09F0E06017F6F040E806F60
:106E1400BC0E816F980E826F000E836FA6EC14F087
:106E24009F0E0601706F040E716FC1EC25F0ECEC3F
:106E340027F0EEEC13F0A30E0B6E570E0C6E020E41
:106E44000D6E0D2EFED70C2EFCD70B2EFAD700009C
:106E5400EEEC13F0300E0601706F960E716F000E9B
:106E6400726F08EC2EF0F18C0001E36BE46BF2928C
:106E7400F2889D98580E0601706F960E716F000E81
:106E8400726F08EC2EF0D09EF18C9F8A9F809D8AB1
:106E94009D80F28CF28E0001EA6BEB6BEEEC13F04A
:106EA400AB880001E56BE66B06016C6B6D6B000152
:106EB400E76BE86B000ED76F010ED86F040E636F9B
:106EC400060E646F5DEC2AF063C07FF664C080F642
:106ED400C4EC11F000C043F001C044F063C068F09A
:106EE40064C069F063C07FF664C080F6E1EC11F021
:106EF400EEEC13F09F0E0601706F040E716F180E06
:106F0400726F980E736F000E746F43C075F644C0B1
:106F140076F63FEC25F09F0E7F6F040E806F62ECD7
:106F240014F068C070F669C071F6C1EC25F0F288FF
:106F3400E80E0601706F970E716F000E726F08EC09
:106F44002EF005016B6B6C6B0001E56BE66B63C0A7
:106F540068F064C069F0AF6BB06B05013397000152
:106F6400AF4BB02BDBEC2DF0010E0001AF15016E21
:106F7400B0C002F0000E0216000E021802E1000E6C
:106F84000118D8A49FD0800E0601706F0F0E716F88
:106F9400726BB1EC30F0800E706F0F0E716F726B0C
:106FA400CC0E736FE9EC30F0800E706F0F0E716FC2
:106FB400726B440E736FE9EC30F0D00E0C6EC90E98
:106FC4000D6E0D2EFED70C2EFCD700000000800E97
:106FD400706F0F0E716F726BB1EC30F0800E706FCA
:106FE4000F0E716F726BCC0E736FE9EC30F0800E84
:106FF400706F0F0E716F726BBE0E736FE9EC30F031
:107004002A0E0C6E8D0E0D6E0D2EFED70C2EFCD797
:1070140000000000800E706F0F0E716F726BF0EC49
:107024002EF000C047F0000E486E800E706F0F0EF9
:10703400716F726BF0EC2EF000C003F0026A4750DF
:107044000224006E48500320016E00C045F001C0C8
:1070540046F0640E046E000E056E99EC10F000C04C
:1070640002F001C003F003320232039E0332023203
:10707400039E03320232039E03320232039E02C095
:107084006DF503C06EF50001CF510224006ED0519E
:107094000320016E00C06DF501C06EF500C070F6EE
:1070A40001C071F6710E0601726F050E736FBFECAD
:1070B4002CF00501786B76C577F575C576F52E0E3F
:1070C400756F0CD0020E0B6E380E0C6EAD0E0D6E7D
:1070D4000D2EFED70C2EFCD70B2EFAD763C07FF6ED
:1070E40064C080F6C4EC11F000C043F001C044F069
:1070F40063C068F064C069F0800E006E800E050104
:107104006C19005C02E16B510708D8B0D3D06B6BEB
:107114006C6B0001E551435C05016F6F0001E651A2
:1071240044580501706F6F4B702B0C0E435C016E5D
:10713400000E4458026E800E0001E619006E800EA7
:107144000218005C02E10150E55D26E20501666B70
:10715400676B800E6719006E800E005C02E10C0EF6
:10716400665D19E29F0E6625E16E010E6721E26EEF
:107174000001E5516825006EE6516921016E0501A3
:1071840066510024E96E67510120EA6EEECFE6FFF6
:10719400664B672BDED74ED00501666B676B800E9E
:1071A4006719006E800E7019005C02E16F51665D14
:1071B40019E29F0E6625E16E010E6721E26E000161
:1071C400E5516825006EE6516921016E050166519D
:1071D4000024E96E67510120EA6EEECFE6FF664BAC
:1071E400672BDDD76FC566F570C567F5800E671927
:1071F400006E800E005C02E10C0E665D1BE29F0EC9
:107204006625E16E010E6721E26E66510001682574
:10721400006E0501675100016921016E05016F517E
:10722400005CE96E70510158EA6EEECFE6FF664BE2
:10723400672BDCD7800E4418006E800E0001E6191F
:10724400005C02E1E551435C2BE2E56BE66B040E66
:10725400636F060E646F63C068F064C069F0050173
:10726400666B676B800E6719006E800E005C02E12E
:107274000C0E665D15E29F0E6625E16E010E672118
:10728400E26E665100016825E96E0501675100014F
:107294006921EA6EEECFE6FF0501664B672BE2D764
:1072A4009F0E0601706F010E716FC1EC25F0000195
:1072B400E54BE62BECEC27F02DEC2DF081A40CD063
:1072C400050E0B6E0F0E0C6EF10E0D6E0D2EFED70D
:1072D4000C2EFCD70B2EFAD70501666B676B0001E9
:1072E40066510501675D04E1000165510501665DB4
:1072F4000CE2150E0C6EC60E0D6E0D2EFED70C2E66
:10730400FCD70000664B672BEAD76B4B6C2B000E47
:107314000001CD1902E1010ECC19D8A4FFEF41F010
:10732400F29EA00E06016C6F050E6D6F6CC6E9FF30
:107334006DC6EAFFEE50480A67E1030E6C25E96E5C
:10734400000E6D21EA6EEE50700A5EE1010E706F60
:10735400980E716F000E726F08EC2EF0E00E0601AD
:10736400706F950E716F000E726F08EC2EF0310E77
:107374000601706F950E716F000E726F08EC2EF09F
:107384008B0E0601706F950E716F000E726F08EC14
:107394002EF0CF0E0601706F930E716F000E726F98
:1073A40008EC2EF0A90E0601706F8F0E716F000E9F
:1073B400726F08EC2EF0010E0601706F900E716F63
:1073C400000E726F08EC2EF03A0E0601706F920EEA
:1073D400716F000E726F08EC2EF07A0E0601706F5A
:1073E400920E716F000E726F08EC2EF0EC0E060117
:1073F400706F900E716F000E726F08EC2EF0EEEC51
:1074040013F006016C6B6D6B6CC6E9FF6DC6EAFF89
:10741400EE50550A42E1140E6C25E96E000E6D2102
:10742400EA6EEE50230A0AE0140E6C25E96E000E93
:107434006D21EA6EEE503B0A01E02FD0580E706FBA
:10744400980E716F000E726F08EC2EF0A00E0601FC
:107454007F6F050E806F62EC14F0EEEC13F0C6EC57
:1074640028F0FAEC29F068C57FF6E2EC24F000C0BD
:1074740065F5FEC07FF6E2EC24F000C06AF5EDC0CD
:107484007FF6E2EC24F000C069F5FBC07FF6E2EC85
:1074940024F000C0ECF06C6B6D6B6CC6E9FF6DC63C
:1074A400EAFFEE504D0A6EE1010E6C25E96E000E06
:1074B4006D21EA6EEE50730A65E1020E6C25E96EE9
:1074C400000E6D21EA6EEE50670A5CE1030E6C2536
:1074D400E96E000E6D21EA6EEE503D0A53E105019E
:1074E400E36B0401EF6BEF0E06017F6F040E806FF8
:1074F400A40E816F050E826F38EC13F0EF0E7F6FD0
:10750400040E806FC4EC11F000C0EAF001C0EBF08F
:10751400000E026E0150025C02E10050030822E2F8
:10752400D90E706F980E716F000E726F08EC2EF00A
:10753400050E0B6E0F0E0C6EF10E0D6E0D2EFED79A
:107544000C2EFCD70B2EFAD700016751000807E276
:1075540067C062F0623762916237629102D0080EAE
:10756400626F0DD0C30E0601706F960E716F000E20
:10757400726F08EC2EF00001626B0401EF6B0601E0
:107584006C6B6D6B6CC6E9FF6DC6EAFFEE50540A76
:10759400D8A4ACD0010E6C25E96E000E6D21EA6E04
:1075A400EE50450AD8A4A2D0020E6C25E96E000E56
:1075B4006D21EA6EEE50780AD8A498D0030E6C259B
:1075C400E96E000E6D21EA6EEE503D0AD8A48ED00D
:1075D4001A6A6CC67FF66DC680F662EC14F06CC64F
:1075E4007FF66DC680F6C4EC11F000C0EAF001C06D
:1075F400EBF00B0E6C25E16E000E6D21E26EE66A77
:10760400050E6C25E96E000E6D21EA6EEECFA7F62D
:107614008DEC10F000C06EF6060E6C25E96E000EBF
:107624006D21EA6EEECFA7F68DEC10F000506E27B8
:107634006F6B000E6F23080E6C25E96E000E6D2132
:10764400EA6EEECFA7F68DEC10F000506E27000E18
:107654006F23090E6C25E96E000E6D21EA6EEECFE4
:10766400A7F68DEC10F000506E250501916F000E09
:1076740006016F210501926F050E06016C25E96E66
:10768400000E6D21EA6EEE50300A08E1050E6C25FD
:10769400E16E000E6D21E26E200EE66E000E050115
:1076A400921902E1040E911915E1000E006E000119
:1076B400EB51005C02E1EA510A080CE2610E06019A
:1076C4007F6F010E806F6CC681F66DC682F638EC52
:1076D40013F009D00601040E7F6F970E806F000E21
:1076E400816FF7EC24F006016C6B6D6B6CC6E9FFDF
:1076F4006DC6EAFFEE50530AD8A422D1010E6C25C0
:10770400E96E000E6D21EA6EEE50700AD8A418D10D
:10771400020E6C25E96E000E6D21EA6EEE50650ACC
:10772400D8A40ED1030E6C25E96E000E6D21EA6E0D
:10773400EE50650AD8A404D1040E6C25E96E000E3F
:107744006D21EA6EEE50640AD8A4FAD0050E6C25B9
:10775400E96E000E6D21EA6EEE503D0AD8A4F0D019
:10776400A00E7F6F050E806F62EC14F0090EAD6FF2
:10777400DAEC00F0CB0E0601706F980E716F000EFC
:10778400726F08EC2EF065C07FF666C080F69F0E1F
:107794000601816F040E826F5FEC13F09F0E7F6F02
:1077A400040E806F62EC14F0090EAD6FDAEC00F099
:1077B400060E06016C25E96E000E6D21EA6EEECF11
:1077C400A7F68DEC10F000C06EF6070E6C25E96E7E
:1077D400000E6D21EA6EEECFA7F68DEC10F000508E
:1077E4006E276F6B000E6F236EC691F56FC692F510
:1077F400060E6C25E96E000E6D21EA6E300EEE5C0D
:10780400006E016A000E015A0A0E046E000E056E27
:1078140099EC10F0070E6C25D96E000E6D21DA6E0E
:10782400DE5000240001EA6F000E0120EB6F300EE1
:10783400EA5F000EEB5B000E06016F1902E1020E17
:107844006E1972E1000E0001EB5D02E1040EEA5DC7
:107854006BE3000EEB5D02E1630EEA5D65E2EAC0F4
:1078640065F0EBC066F0A60E0601706F000E716F36
:107874000A0E046E000E056EEAC000F0EBC001F0C3
:10788400C1EC10F0300E0024726F3CEC2AF0030EB1
:107894000B6E080E0C6E770E0D6E0D2EFED70C2E91
:1078A400FCD70B2EFAD7A70E0601706F000E716F6E
:1078B4000A0E046E000E056EEAC000F0EBC001F083
:1078C400C1EC10F008C000F009C001F0300E002433
:1078D400726F3CEC2AF0030E0B6E080E0C6E770EE2
:1078E4000D6E0D2EFED70C2EFCD70B2EFAD7C20E22
:1078F4000601706F990E716F000E726F08EC2EF016
:10790400A00E0601706F000E716F9F0E726F040E51
:10791400736F2BEC2EF09F0E7F6F040E806F62EC62
:1079240014F0EEEC13F009D0030E0601706F950EFF
:10793400716F000E726F08EC2EF006016C6B6D6BAC
:107944006CC6E9FF6DC6EAFFEE504C0AD8A40DD10F
:10795400010E6C25E96E000E6D21EA6EEE50750A7B
:10796400D8A403D1020E6C25E96E000E6D21EA6ED7
:10797400EE506D0AD8A4F9D0030E6C25E96E000E02
:107984006D21EA6EEE503D0AD8A4EFD0A00E7F6FB1
:10799400050E806F62EC14F0090EAD6FDAEC00F0A6
:1079A400310E0601706F990E716F000E726F08EC44
:1079B4002EF019C07FF6000E0601806F9F0E816FB6
:1079C400040E826F5FEC13F09F0E7F6F040E806FC6
:1079D40062EC14F0090EAD6FDAEC00F0040E06014F
:1079E4006C25E96E000E6D21EA6EEECFA7F68DECE4
:1079F40010F000C06EF6050E6C25E96E000E6D21C8
:107A0400EA6EEECFA7F68DEC10F000506E276F6B88
:107A1400000E6F236EC691F56FC692F5040E6C25A9
:107A2400E96E000E6D21EA6E300EEE5C006E016AA6
:107A3400000E015A0A0E046E000E056E99EC10F049
:107A4400050E6C25D96E000E6D21DA6EDE50002411
:107A54000001EA6F000E0120EB6F300EEA5F000EAA
:107A6400EB5B000E06016F1902E1020E6E1971E163
:107A7400000E0001EB5D02E1000EEA5D6AE3000E18
:107A8400EB5D02E10B0EEA5D64E20F0EEA15196E7E
:107A9400C40E0601706F000E716F0A0E046E000EA4
:107AA400056EEAC000F0EBC001F0C1EC10F0300E3E
:107AB4000024726F3CEC2AF0030E0B6E080E0C6E61
:107AC400770E0D6E0D2EFED70C2EFCD70B2EFAD78B
:107AD400C50E0601706F000E716F0A0E046E000E63
:107AE400056EEAC000F0EBC001F0C1EC10F008C074
:107AF40000F009C001F0300E0024726F3CEC2AF053
:107B0400030E0B6E080E0C6E770E0D6E0D2EFED747
:107B14000C2EFCD70B2EFAD7DA0E0601706F990ED5
:107B2400716F000E726F08EC2EF0C00E0601706FBC
:107B3400000E716F9F0E726F040E736F2BEC2EF09C
:107B44009F0E7F6F040E806F62EC14F0EEEC13F066
:107B540009D05E0E0601706F950E716F000E726F84
:107B640008EC2EF006016C6B6D6B6CC6E9FF6DC6FC
:107B7400EAFFEE50520AD8A4C5D0010E6C25E96E76
:107B8400000E6D21EA6EEE50650AD8A4BBD0020E39
:107B94006C25E96E000E6D21EA6EEE50700AD8A4D1
:107BA400B1D0030E6C25E96E000E6D21EA6EEE5025
:107BB4003D0AD8A4A7D0A00E7F6F050E806F62EC9B
:107BC40014F0090EAD6FDAEC00F00E0E0601706FC2
:107BD400990E716F000E726F08EC2EF067C07FF67D
:107BE400000E0601806F9F0E816F040E826F5FECA2
:107BF40013F09F0E7F6F040E806F62EC14F0090E79
:107C0400AD6FDAEC00F0040E06016C25E96E000E8F
:107C14006D21EA6EEECFA7F68DEC10F000C06EF683
:107C2400050E6C25E96E000E6D21EA6EEECFA7F607
:107C34008DEC10F000506E276F6B000E6F236EC634
:107C440091F56FC692F5040E6C25E96E000E6D2158
:107C5400EA6E300EEE5C006E016A000E015A0A0EE6
:107C6400046E000E056E99EC10F0050E6C25D96EAD
:107C7400000E6D21DA6EDE5000240001EA6F000E62
:107C84000120EB6F300EEA5F000EEB5B000E060185
:107C94006F1902E1020E6E1902E1EAC067F0040EE8
:107CA4000001675D20E3675132081DE31A0E0601E7
:107CB400706F990E716F000E726F08EC2EF067C032
:107CC4007FF6000E0601806F9F0E816F040E826F97
:107CD4005FEC13F09F0E7F6F040E806F62EC14F064
:107CE400EEEC13F00CD0040E0001676FB60E060123
:107CF400706F950E716F000E726F08EC2EF0060116
:107D04006C6B6D6B6CC6E9FF6DC6EAFFEE50500AF2
:107D1400D8A4A9D1010E6C25E96E000E6D21EA6E7E
:107D2400EE504C0AD8A49FD1020E6C25E96E000EC9
:107D34006D21EA6EEE504D0AD8A495D1030E6C2540
:107D4400E96E000E6D21EA6EEE503D0AD8A48BD187
:107D5400A00E7F6F050E806FC4EC11F0800E011829
:107D6400026E800E025C02E1090E005CD8A07BD199
:107D7400A00E7F6F050E806F62EC14F0090EAD6FDC
:107D8400DAEC00F0060E06016C25E16E000E6D21A2
:107D9400E26EE66A090E6C25E16E000E6D21E26E5C
:107DA400E66A9A0E706F990E716F000E726F08EC8E
:107DB4002EF0900E0601706F000E716F9F0E726FA1
:107DC400040E736F2BEC2EF09F0E7F6F040E806FEA
:107DD40062EC14F0090EAD6FDAEC00F0040E06014B
:107DE4006C25E96E000E6D21EA6EEECFA7F68DECE0
:107DF40010F000C06EF6050E6C25E96E000E6D21C4
:107E0400EA6EEECFA7F68DEC10F000506E276F6B84
:107E1400000E6F23070E6C25E96E000E6D21EA6ECD
:107E2400EECFA7F68DEC10F000506E27000E6F23F6
:107E3400080E6C25E96E000E6D21EA6EEECFA7F6F2
:107E44008DEC10F000506E27000E6F236EC691F576
:107E54006FC692F5040E6C25E96E000E6D21EA6E74
:107E6400300EEE5C006E016A000E015A0A0E046EBA
:107E7400000E056E99EC10F0050E6C25D96E000EFF
:107E84006D21DA6EDE5000240001EA6F000E01203D
:107E9400EB6F300EEA5F000EEB5B070E06016C25FC
:107EA400E96E000E6D21EA6E300EEE5C006E016A22
:107EB400000E015A0A0E046E000E056E99EC10F0C5
:107EC400080E6C25D96E000E6D21DA6EDE5000248A
:107ED4000501966F000E0120976F300E965F000E1D
:107EE400975B000E06016F1902E1040E6E19D8A407
:107EF400ACD0000E006E0001EB51005C02E1EA51CF
:107F04000C08D8B0A2D0000EEB5D02E1180EEA5DB9
:107F1400D8B09BD0000E0501975D02E1000E965D7E
:107F2400D8A093D0000E975D02E10C0E965DD8B0F8
:107F34008CD0EAC0DAF0040E06016C25E96E000E5E
:107F44006D21EA6EEECFCEF0940E706F000E716F5D
:107F5400CEC072F63CEC2AF0050E06016C25E96EE3
:107F6400000E6D21EA6EEECFCEF0950E706F000E0E
:107F7400716FCEC072F63CEC2AF0030E0B6E080E45
:107F84000C6E770E0D6E0D2EFED70C2EFCD70B2E1D
:107F9400FAD796C5D9F0070E06016C25E96E000ED6
:107FA4006D21EA6EEECFCEF0970E706F000E716FFA
:107FB400CEC072F63CEC2AF0030E0B6E080E0C6E6B
:107FC400770E0D6E0D2EFED70C2EFCD70B2EFAD786
:107FD400080E06016C25E96E000E6D21EA6EEECFE7
:107FE400CEF0980E706F000E716FCEC072F63CEC3E
:107FF4002AF0030E0B6E080E0C6E770E0D6E0D2E0E
:10800400FED70C2EFCD70B2EFAD7900E0601706FFC
:10801400000E716F9F0E726F040E736F2BEC2EF0B7
:10802400030E0B6E080E0C6E770E0D6E0D2EFED722
:108034000C2EFCD70B2EFAD79F0E7F6F040E806F89
:1080440062EC14F0EEEC13F009D02B0E0601706F05
:10805400930E716F000E726F08EC2EF0EEEC13F0BD
:1080640006016C6B6D6B6CC6E9FF6DC6EAFFEE50E2
:10807400430AD8A4BED1010E6C25E96E000E6D2111
:10808400EA6EEE504F0AD8A4B4D1020E6C25E96E04
:10809400000E6D21EA6EEE50520AD8A4AAD1040E45
:1080A4006C25E96E000E6D21EA6EEE503D0AD8A4EF
:1080B400A0D16CC67FF66DC680F6C4EC11F0800EBC
:1080C4000118026E800E025C02E1090E005CD8A069
:1080D40090D1E20E706F990E716F000E726F08EC02
:1080E4002EF06CC67FF66DC680F662EC14F0090EB5
:1080F400AD6FDAEC00F00A0E06016C25E16E000E9D
:108104006D21E26EE66AB20E706F990E716F000E09
:10811400726F08EC2EF0030E06016C25E96E000E5A
:108124006D21EA6EEE50310A05E1D00E0501946F1F
:10813400000E956F030E06016C25E96E000E6D218D
:10814400EA6EEE50320A05E1E00E0501946F000E6E
:10815400956F94C570F695C571F69F0E0601726F02
:10816400040E736F2BEC2EF09F0E7F6F040E806F46
:1081740062EC14F0060E6C25E96E000E6D21EA6EB9
:10818400EECFA7F68DEC10F000C06EF6070E6C254E
:10819400E96E000E6D21EA6EEECFA7F68DEC10F0BD
:1081A40000506E276F6B000E6F23080E6C25E96E6E
:1081B400000E6D21EA6EEECFA7F68DEC10F00050A4
:1081C4006E25016E000E6F21026E01C091F502C092
:1081D40092F5000E021802E1030E0118D8A406D18C
:1081E400050E6C257F6F000E6D21806FF9EC13F086
:1081F40000C098F501C099F5800E0118026E800E3A
:10820400010A025C02E12C0E005CD8B0E6D0800EBC
:10821400FE0A006E800E05019919005C02E1985176
:10822400D408D8B0DAD0030E06016C25E96E000E2E
:108234006D21EA6EEE50310A0AE0030E6C25E96EF8
:10824400000E6D21EA6EEE50320A01E0C5D0030E35
:108254006C25E96E000E6D21EA6EEE50310A21E1C3
:10826400D00E0501946F000E956F98C5CFF099C597
:10827400D0F098C500F099C501F0CFEC2EF0000EB7
:10828400046E000E056E480E066E850E076E84ECB5
:1082940006F000C0D1F001C0D2F002C0D3F003C098
:1082A400D4F0030E06016C25E96E000E6D21EA6E12
:1082B400EE50320A21E1E00E0501946F000E956F35
:1082C40098C59EF599C59FF598C500F099C501F02C
:1082D400CFEC2EF0000E046E000E056E480E066EF6
:1082E400850E076E84EC06F000C09AF501C09BF57C
:1082F40002C09CF503C09DF50501306B316B000E87
:10830400315D02E1040E305D32E2050E9425060172
:10831400706F000E050195210601716F0501305142
:10832400060170270501315106017123050E6C25E4
:10833400006E000E6D21016E050130510024E96EBE
:1083440031510120EA6EEECF72F63CEC2AF0030EB6
:108354000B6E080E0C6E770E0D6E0D2EFED70C2EC6
:10836400FCD70B2EFAD70501304B312BC8D7AA0EF8
:108374000601706F990E716F000E726F08EC2EF08B
:108384006CC6E9FF6DC6EAFF030EEE240601AD6F6D
:10839400DAEC00F03A0E0601AD6FDAEC00F094C5A9
:1083A40070F695C571F69F0E0601726F040E736F19
:1083B4002BEC2EF0030E0B6E080E0C6E770E0D6E6A
:1083C4000D2EFED70C2EFCD70B2EFAD79F0E7F6FE7
:1083D400040E806F62EC14F009D00601A20E706FD7
:1083E400940E716F000E726F08EC2EF006016C6B28
:1083F4006D6B0001CC6BCD6BF28E000EE41902E1C3
:10840400000EE319D8B47EEF38F0E36BE46B1A2A5C
:108414001A503C080DE2610E06017F6F010E806F59
:10842400E70E816F980E826F000E836FA6EC14F036
:10843400F28800016251000808E262076251000AF2
:1084440004E17AEC25F00401EF6B0601706B9DECFE
:1084540026F0040E0001636F060E646F5DEC2AF0D3
:10846400616B300EB15D006E0A0E0002F3CF01F0B5
:10847400300EB25D006E0050012601C093F5D95153
:10848400015C07E3DA510501935D03E2010E00018B
:10849400616F000E0501935D07E30001D9510501E9
:1084A400935D02E20001616B00016151000A12E177
:1084B4000A0E06017F6F806B816B826B836B846B0A
:1084C400856B866B876B886B896B8A6B8B6B14EC03
:1084D40011F01DD00A0E06017F6F19C080F619C075
:1084E40081F619C082F619C083F619C084F619C042
:1084F40085F619C086F619C087F619C088F619C022
:1085040089F619C08AF619C08BF614EC11F0897833
:06851400B1EF37F0FFD7C4
:109A300010EE19F0B60E006E010E016E1A0EF66EE3
:0E9A40008D0EF76E000EF86E64EC25F012002D
:10851A0000000000000000007E81A581BD99817ED7
:10852A007EFFDBFFC3E7FF7E6CFEFEFE7C38100099
:10853A0010387CFE7C381000383838FEFED61038E9
:10854A001010387CFE7C10380000183C3C180000E3
:10855A00FFFFE7C3C3E7FFFF003C664242663C00F9
:10856A00FFC399BDBD99C3FF0F03057D8484847839
:10857A003C4242423C187E183F213F202060E0C026
:10858A003F213F212367E6C018DB3CE7E73CDB18C5
:10859A0080E0F8FEF8E08000020E3EFE3E0E020089
:1085AA00183C7E18187E3C18242424242400240015
:1085BA007F929272121212003E6338444438CC7889
:1085CA00000000007E7E7E00183C7E187E3C18FF6C
:1085DA0010387C5410101000101010547C38100001
:1085EA0000180CFE0C180000003060FE603000001D
:1085FA0000004040407E0000002466FF6624000020
:10860A000010387CFEFE000000FEFE7C38100000E0
:10861A0000000000000000001010101010001000F0
:10862A00242424000000000024247E247E24240024
:10863A00183E403C027C180000626408102646007E
:10864A00304830568888760010102000000000005C
:10865A001020404040201000201008080810200078
:10866A00004438FE384400000010107C101000004E
:10867A0000000000001010200000007E0000000032
:10868A000000000000101000000204081020400042
:10869A003C42464A52623C001030501010107C0096
:1086AA003C42020C30427E003C42021C02423C0028
:1086BA0008182848FE081C007E407C0202423C0042
:1086CA001C20407C42423C007E42040810101000EC
:1086DA003C42423C42423C003C42423E0204380098
:1086EA0000101000001010000010100000101020E0
:1086FA00081020402010080000007E00007E0000C4
:10870A0010080402040810003C4202040800080091
:10871A003C425E525E403C00182442427E42420085
:10872A007C22223C22227C001C22404040221C0047
:10873A0078242222222478007E22283828227E00C9
:10874A007E222838282070001C2240404E221E001B
:10875A004242427E42424200381010101010380045
:10876A000E04040444443800622428302824630098
:10877A007020202020227E0063554941414141005A
:10878A0062524A46424242003C42424242423C0013
:10879A007C22223C202070003C4242424A3C030098
:1087AA007C22223C282472003C42403C02423C008B
:1087BA007F49080808081C004242424242423C00E3
:1087CA004141414122140800414141494949360089
:1087DA0041221408142241004122140808081C00EE
:1087EA007F42040810217F007840404040407800D2
:1087FA008040201008040200780808080808780059
:10880A00102844820000000000000000000000FF61
:10881A00101008000000000000003C023E423F0029
:10882A006020202E31312E0000003C4240423C00A4
:10883A000602023A46463B0000003C427E403C00AB
:10884A000C1210381010380000003D42423E027CE3
:10885A0060202C32222262001000301010103800E2
:10886A00020006020242423C6020242830282600E8
:10887A00301010101010380000007649494949009C
:10888A0000005C624242420000003C4242423C001C
:10889A0000006C32322C20700000364C4C34040E2E
:1088AA0000006C322220700000003E403C027C0036
:1088BA0010107C1010120C000000424242463A008E
:1088CA00000041412214080000004149494936008C
:1088DA00000044281028440000004242423E027C24
:1088EA0000007C0810207C000C10106010100C0096
:1088FA001010100010101000300808060808300088
:10890A00324C0000000000001C14141C000000007F
:10891A003C4240423C0C023C0044004444443E0079
:10892A000C003C427E403C003C4238043C443E0041
:10893A00420038043C443E00300038043C443E00C7
:10894A003C2424243C00000000003C40403C061C1F
:10895A003C423C427E403C0042003C427E403C005D
:10896A0030003C427E403C002400180808081C00E5
:10897A007C823010101038003000180808081C00DB
:10898A00421824427E4242001818003C427E4200AD
:10899A000C007C2038207C000000330C3F443B0054
:1089AA001F24447F444447001824003C42423C00B0
:1089BA000042003C42423C002010003C42423C0043
:1089CA001824004242423C002010004242423C002D
:1089DA0000420042423E023C42182442422418000D
:1089EA004200424242423C0008083E40403E0808DB
:1089FA001824207020427C0044287C107C1010002F
:108A0A00F84C78444F4445E61C12107C10109060D4
:108A1A000C0038043C443E000C00180808081C00EE
:108A2A000408003C42423C000004084242423C0026
:108A3A00324C007C42424200324C0062524A4600AA
:108A4A003C44443E007E000038444438007C000028
:108A5A001000102040423C000000007E4040000010
:108A6A000000007E0202000042C448F629438C1F1F
:108A7A0042C44AF62A5F8202001000101010100049
:108A8A00001224482412000000482412244800003E
:108A9A00228822882288228855AA55AA55AA55AA28
:108AAA00DB77DBEEDB77DBEE101010101010101006
:108ABA0010101010F01010101010F010F01010100C
:108ACA0014141414F414141400000000FC141414E4
:108ADA000000F010F01010101414F404F41414141C
:108AEA0014141414141414140000FC04F4141414AC
:108AFA001414F404FC00000014141414FC00000004
:108B0A001010F010F000000000000000F01010102B
:108B1A00101010101F00000010101010FF000000AD
:108B2A0000000000FF101010101010101F1010107D
:108B3A0000000000FF00000010101010FF101010BD
:108B4A0010101F101F1010101414141417141414DA
:108B5A00141417101F00000000001F10171414141B
:108B6A001414F700FF0000000000FF00F7141414AB
:108B7A0014141710171414140000FF00FF0000004B
:108B8A001414F700F71414141010FF00FF0000006B
:108B9A0014141414FF0000000000FF00FF1010104E
:108BAA0000000000FF141414141414141F00000011
:108BBA0010101F101F00000000001F101F101010BF
:108BCA00000000001F14141414141414FF141414B5
:108BDA001010FF10FF10101010101010F0000000FD
:108BEA00000000001F101010FFFFFFFFFFFFFFFF34
:108BFA0000000000FFFFFFFFF0F0F0F0F0F0F0F0EF
:108C0A000F0F0F0F0F0F0F0FFFFFFFFF00000000E6
:108C1A000000314A444A3100003C427C427C4040D8
:108C2A00007E424040404000003F54141414140097
:108C3A007E42201820427E0000003E48484830000C
:108C4A00004444447A40408000334C080808080035
:108C5A007C1038444438107C1824427E4224180080
:108C6A0018244242242466001C20183C42423C003C
:108C7A00006295899562000002043C4A523C408099
:108C8A000C10203C20100C003C424242424242005E
:108C9A00007E007E007E000010107C1010007C0018
:108CAA001008040810007E000810201008007E003A
:108CBA000C1212101010101010101010109090605A
:108CCA001818007E0018180000324C00324C0000C0
:108CDA00304848300000000000000018180000006A
:108CEA0000000000180000000F08080808C828182B
:108CFA0078444444440000003048102078000000C2
:108D0A0000003C3C3C3C0000000000000000000069
:018D1A000058
:018D1B000057
:018D1C000155
:108D1D00B49700368E00D08D009B8E00529000F2DD
:108D2D009200AD9800B89100329100518F0075916D
:078D3D0000F78E00A090007A
:028D440000002D
:028D460000002B
:028D4800000029
:108D4A00119A00E99900F09900469900FE99003CB1
:088D5A00990092990064990050
:018D62000010
:018D63000609
:028D6400040603
:028D66006300A8
:018D68000604
:028D69000406FE
:108D6B00A29900809900779900179A00F79900272C
:108D7B009A00059A006E99000B9A00269900899922
:078D8B00005A990050990005
:028D92000000DF
:028D94000000DD
:028D96000000DB
:028D98000000D9
:028D9A000000D7
:048D9C0000000000D3
:078DA000286E756C6C2900C0
:098DA70030302F30302F30300045
:028DB0000000C1
:098DB20030303A30303A30300024
:028DBB000000B6
:028DBD000000B4
:028DBF000000B2
:028DC1000000B0
:088DC30070507704040404075A
:028DCB000000A6
:028DCD000000A4
:018DCF0000A3
:108DD0002050726F6A6574203A20486F726C6F671A
:108DE000655F323032305F446566696C5F31325F97
:108DF0004D6174726963653878385F485F393662EF
:108E00006974735F4453333233315F4453313842B2
:108E100032305F484330355F31384632364B32327C
:108E20005F524E34315F323032305F30382E6D63F6
:068E30007070690D0A00DC
:108E3600204469726563746F7279203A20433A5C04
:108E46005F4D696B726F435C5F4D657350726F6AFD
:108E56006574735F4D696B726F435C486F726C6FBC
:108E660067655F31326D617472696365735F387807
:108E7600385F646566696C745F3936626974735FFE
:108E860061736D5F31384632364B32325F32303283
:058E960030200D0A0070
:108E9B0020536F75726365203A20486F726C6F6751
:108EAB00655F323032305F646566696C5F31325FAB
:108EBB004D617472696365735F3878385F393662F8
:108ECB006974735F31384632364B32325F31784FCB
:108EDB0057535F484330355F524E34315F32303237
:0C8EEB00305F303830352E63200D0A0057
:108EF700205049432045656570726F6D203A2048C0
:108F07006F726C6F67655F323032305F44656669D8
:108F17006C5F31325F4D6174726963653878385FB1
:108F2700485F3936626974735F31384632364B327F
:108F3700325F323032305F303730395F454550521B
:0A8F47004F4D2E696865780D0A0091
:108F51002044657669636573203A20332078203494
:108F6100204D4158373231392028636D732920480B
:108F71006F72697A6F6E74616C20636F6E6E656378
:108F8100746564202C525443204453333233312CC2
:108F9100203178204F575320445331384232302CFE
:088FA10020484330350D0A00A1
:108FA900204D73673D782E2E2E7820646520302061
:108FB900E0203633206361726163746572657320E2
:108FC9002C207369203E30202C2041666669636835
:108FD90065206C65206D65737361676520782E2E39
:108FE9002E782070656E64616E74207820526570E9
:088FF900203C43523E0D0A002A
:1090010020657420616666696368616765205469DB
:109011006D65207265647569742C207061732064BC
:1090210027696E666F2074656D7065726174757203
:1090310065732070656E64616E74206C65204D737C
:109041006720416666696368E9203C43523E0D0A28
:01905100001E
:1090520020557361676520646520382072656769F1
:109062007374726573206465203936206269747383
:109072002028332078206C6F6E672920706F7572FC
:1090820020646563616C61676520E02067617563D8
:0E9092006865202E2E656E2041534D0D0A009C
:1090A000204D65732E2054656D706572204578746F
:1090B00065722064697374616E74652076696120DD
:1090C00050494331324631383430206574204843AA
:1090D0003132206D6F64652046553220343830308F
:0C90E0002063616E616C2031340D0A00C9
:1090EC002054656D702E45787465726965757220B3
:1090FC003A20636170746575722067E972E92070BB
:10910C00617220504943313246313834302C20655D
:10911C006E766F692076696120626C7565746F6F0D
:06912C007468200D0A002A
:1091320020436F6E666967204F7363696C6C61745C
:10914200657572203A2050494331384632366B32C7
:10915200325F464F53435F696E7465726E655F316D
:109162003678342D36344D485A2E636667736368F9
:039172000D0A00E3
:109175002050726F746F636F6C6573203A202053B3
:109185005049206269742062616E672C2049324320
:10919500312048617264776172652C2055415254C3
:1091A500312048617264776172652C204F575320D6
:0391B5000D0A00A0
:1091B8002054696E795F5254435F445333323331DC
:1091C8005F666F725F4149325F323032302E6D63B5
:1091D8006C206574202A2E68202C466F6E74203A05
:1091E800205468696E5F53535F323032302E480D19
:0291F8000A006B
:1091FA0020553A30333B31323B31393B31383B33FE
:10920A00363B30322020706F75722030332064650F
:10921A0063656D62726520323031392020313848F9
:10922A0033362030323D4D617264690D0A0D0A00F1
:10923A00205265703D787820646520303420E02023
:10924A003939203A52657065746974696F6E2064A1
:10925A0075204D73672070656E64616E742078782E
:10926A00204379636C657320203C43523E0D0A000B
:10927A00204C756D3D787820646520303020E020E0
:10928A003135203A5265676C616765204C756D69A6
:10929A006E6F736974E920656E206D6F6465204A8C
:0C92AA004F555220203C43523E0D0A005C
:1092B600204269742042616E6720536F66742053A2
:1092C600504920205243323D436C6B202C5243318F
:1092D6003D446F757420205243303D4353202D3E4C
:0C92E600204D4178373231393A0D0A0032
:1092F200205465726D696E616C20706F75722064A6
:1093020069616C6F67756520657420566973752095
:10931200206465726F756C656D656E742070726F16
:099322006772616D6D650D0A00B2
:10932B002042414420504C4D2076616C7565732171
:10933B00206D7573742062652066726F6D205B31D2
:10934B00332E2E203233205D20746F205B20302093
:08935B002E2E203131205D00AF
:109363002041666669636861676520427566666564
:109373007220646570756973203C4F4646534554AB
:109383003D3078313030683E203234206C6F6E6768
:069393007321200D0A0009
:109399002054657374204166666963686167652056
:1093A9005354415449515545206465203132206355
:1093B900617273203A3C30313233343536373839BB
:0693C90041423E0D0A00C6
:1093CF002053706565643D787820207669746573E5
:1093DF00736520646520646566696C656D656E7480
:1093EF0020787820646520303220E0203939203C05
:0693FF0043523E0D0A007E
:109405000D0A2052617070656C20666F726D617413
:1094150020646520636465203A2022553B4A4A3B17
:109425004D4D3B41413B48483B4D4D3B6A443B23F9
:0594350022200D0A00D9
:10943A000000007F000020820000488500007A8832
:10944A0000401C8C0050438F00247492809618961A
:10945A0020BC3E99286B6E9CF90215A0EC782DC1B0
:04946A00CAF249E217
:10946E000000007FCDCC4C7B0AD723786F1203759A
:10947E0017B75171ACC5276EBD37066B95BF5667D2
:10948E0077CC2B645F700961FFE65B5D08E53C3CC1
:04949E006042221BEB
:1094A2002042414420434F52782076616C756520FA
:1094B2006D75737420696E207468652072616E67C1
:1094C20065203C2D33303020746F202B3330305DDB
:0194D2000099
:1094D300010000000800000040000000000200003E
:1094E30000100000008000000000040000002000C5
:1094F3000000000100000008000000400000000020
:10950300204241442053706565642076616C756523
:1095130021206D75737420626520626574776565BB
:0E9523006E20303520616E642039380D0A004C
:10953100206578656D706C6520706F7572203A31A9
:1095410034204D61692032303138203031284C755A
:0D9551006E6469292031354833360D0A005B
:10955E0020424144204C756D2076616C756520214A
:10956E00206D757374206265206265747765656E13
:0D957E0020303020616E642031300D0A0075
:10958B0020506C616765204C756D696E6F736974E3
:10959B00E9204D696E696D616C6520504C4D3D3114
:0B95AB00383A30363C43523E0D0A00B7
:1095B60020424144205265702076616C75652120F9
:1095C6006D757374206265747765656E202030341E
:0A95D60020616E642035300D0A009C
:1095E00020525443205570646174653A20553B31D4
:1095F000343B30353B31383B31353B33363B303112
:08960000233C43523E0D0A0019
:10960800010000000A00000064000000E8030000F8
:1096180010270000A086010040420F0080969800A5
:0896280000E1F50500CA9A3BC0
:1096300020496E697420496E746572727570742069
:109640005242302C2073796E6368726F2031487AF1
:0896500020525443200D0A00D2
:1096580020496E697420496E746572727570742041
:1096680054494D45523120262055415254205258D4
:04967800200D0A00B7
:10967C00205465737420536F6E64652041204F57DE
:10968C00532044533138423230207375722052418A
:04969C00300D0A0083
:1096A0000D0A45727265757220737572204A6F7566
:1096B000722053656D61696E65206A532E204F4B91
:0396C0000D0A0090
:1096C300204D736720646F69742065747265203E52
:1096D30030206574203C36332063617273210D0A98
:0196E3000086
:1096E4000100000010000000000100000010000054
:1096F4000000010000001000000000010000001044
:1097040020424144206D757374206265206C696B3E
:0F97140065205465783D2B32312E33330D0A001A
:1097230020436C656172203132204D61747269632C
:0E9733006573204D415837323139200D0A0040
:1097410020526563757065726520706172616D6527
:0E9751007472657320456570726F6D0D0A00AD
:10975F0045637269747572652064616E732044533A
:0D976F00333233312E2E2E204F4B0D0A00C9
:10977C0020496E6974203132204D617472696365C1
:0D978C0073204D415837323139200D0A004D
:109799002041637469766520736F7274696520531B
:0B97A90051573D31487A3A200D0A006C
:1097B400204D696B726F6320372E362E302031387E
:0A97C4004632364B3232200D0A0007
:1097CE00204D657375726520427275746520445321
:0A97DE0031384232305F413D200077
:1097E8002044656D6D617261676520646563616CB5
:0997F800616765203A200D0A00AA
:109801000D0A2048656C70203A2048656C703C4315
:07981100523E20200D0A0069
:10981800204C6F6E67205472616D65203D202535A0
:069828006420200D0A007F
:10982E0020496E69742052544320445333323331ED
:05983E003A200D0A00B4
:109843002052652D4C656374757265205254432014
:059853002D3E20200065
:109858002043646520525443205570646174652028
:039868003A2000A3
:10986B00303132333435363738396162636465668B
:01987B0000EC
:10987C00303132333435363738394142434445463A
:01988C0000DB
:10988D002046616D696C7920436F6465203A200034
:10989D003031323334353637383941424344454619
:0F98AD0020416C696D203D332E3656200D0A0088
:0F98BC00566572732E323032305F3038303500DF
:0E98CB00204F6C64207370656564203D2000A2
:0E98D900204F4B20666F72204D73670D0A0002
:0D98E700544578204E6F4C696E6B202000B8
:0D98F4000D0A20525443206A53203D2000ED
:0D99010030313233343536373839414200C9
:0C990E00204F6C6420526570203D20004A
:0C991A00204E657720526570203D200033
:0B99260053657074656D62726520006F
:0B993100204F6C64204C756D3D200041
:0A993C0056656E64726564692000D0
:0A9946004D657263726564692000CC
:0A995000446563656D6272652000D6
:0A995A004E6F76656D6272652000A5
:0A99640044696D616E6368652000C0
:09996E004A75696C6C65742000F7
:09997700466576726965722000F4
:099980004A616E766965722000EF
:099989004F63746F6272652000E7
:0899920053616D65646920005A
:08999A00204F6C64203D200009
:0899A2006572726575722E00FA
:0899AA004E657720434F520087
:0899B200204F6C64203D2000F1
:0899BA002031392E3939B000CB
:0899C200204E6577203D2000D6
:0899CA0020204352433D200020
:0899D20020494431203D200032
:0899DA00204E6577203D2000BE
:0799E200204364653A2000F8
:0799E9004C756E646920005B
:0799F0004D61726469200063
:0799F700417672696C20004B
:0799FE004A65756469200051
:069A05004A75696E2000A5
:069A0B00416F757420009C
:069A11006572726F720025
:069A17004D617273200096
:059A1D00B04320200011
:059A220054496E3D00F7
:059A27004D6169200003
:039A2C00202000F7
:020000040030CA
:0D00010078193CFFB781FF0FC00FE00F40E2
:0200000400F00A
:1000000020486F726C6F6765203132204D617472C9
:1000100069636573204820387838202031384632AB
:10002000364B32322020464F53432036344D487AE7
:100030002C2052544320445333323331202C20554A
:10004000415254312031393230302C382C4E2C3141
:100050000D0A204843303520426C7565546F6F742B
:1000600068204573636C6176650D0A0020202020AE
:100070005665722E2032303230303730390D0A005A
:10008000FFFFFFFFFFFFFFFFFFFFFFFFFFFFFFFF80
:10009000504C4D3D32333A30360D0A00202020209E
:1000A00053706565643D31300D0A0020202020200A
:1000B0005265703D30300D0A002020202020202085
:1000C0004C756D3D30310D0A00202020202020206D
:1000D000434F52313D2B3030310D0A00202020207B
:1000E000434F52323D2D3030310D0A002020202068
:1000F000FFFFFFFFFFFFFFFFFFFFFFFFFFFFFFFF10
:10010000FFFFFFFFFFFFFFFFFFFFFFFFFFFFFFFFFF
:10011000FFFFFFFFFFFFFFFFFFFFFFFFFFFFFFFFEF
:10012000FFFFFFFFFFFFFFFFFFFFFFFFFFFFFFFFDF
:1003D0007265762030392F30352F32303230202080
:1003E0007061756C666A756A6F2032303230202019
:1003F00020200D0A00FFFFFFFFFFFFFFFFFFFFFFB1
:00000001FF
